:100000000C94A9030C94D1030C94D1030C94D10348
:100010000C94D1030C94D1030C94D1030C94D10310
:100020000C94D1030C94D1030C94BF300C94622F28
:100030000C94D1030C94D1030C94D1030C94D103F0
:100040000C94D1030C94D1030C94D1030C94D103E0
:100050000C94D1030C94D1030C94D1030C94E703BA
:100060000C94D1030C94D1030C94D1030C94D103C0
:100070000C94D1030C94D1030C94D1030C94D103B0
:100080000C94D1030C94D1030C94D1030C94D103A0
:100090000C94DC320C94D1030C94D1030C94D10356
:1000A0000C94D1030C94D1030C94D1030D8702005E
:1000B000002A01FC0428010E05260120051E023439
:1000C000051B0234051802340515023405120234EA
:1000D000050F0234050C02340524013E052C0149AC
:1000E0000500570537273800000055053701070080
:1000F00000006C6F63616C6C79206275696C7420B0
:100100006F6E2044656320313820323032332061F5
:10011000742031393A34363A3539004B6579626F9B
:10012000617264696F204D6F64656C203031202DE1
:10013000204B616C6569646F73636F70652000FFAD
:10014000FF1E001F002000210022000043E000E409
:10015000000160230024002500260027000144350B
:100160000014001A000800150017002B002A002CAC
:100170000028001C0018000C00120013002E004B79
:100180000004001600070009000A002900E300E24D
:1001900000E6000B000D000E000F00330034004E8F
:1001A000001D001B000600190005002C44E100E5BD
:1001B000002C44110010003600370038002D00FFDD
:1001C000FFFFFFFFFFFFFFFFFFFFFFFFFFFFFFFF3F
:1001D000FF0060FFFF2400250026005600FFFFFF00
:1001E000FFFFFFFFFFFFFFFFFFFFFFFFFFFFFFFF1F
:1001F000FFFFFFFFFF2100220023005700FFFFFF4A
:10020000FFFFFFFFFFFFFFFFFFFFFFFFFFFFFFFFFE
:10021000FFFFFFFFFF1E001F0020002E00FFFFFF5B
:10022000FFFFFFFFFFFFFFFFFFFFFFFFFFFFFFFFDE
:10023000FFFFFFFFFF27003700550054002800FF95
:10024000FF3A003B003C003D003E003900FFFFFF4D
:10025000FFB6483F00400041004200430044002BED
:1002600000FFFF0150FFFF4250605029504C002812
:1002700000CD48B5482F0830082F00300045004A0F
:1002800000045002500850415025502A50FFFFFFF3
:10029000FF65005000510052004F00FFFFFFFF4D6F
:1002A0000046004900FFFF44502650FFFFFFFFFFBC
:1002B000FFFFFFE248EA48E948FFFF31003108301C
:1002C0002E39322E312B39340076657273696F6E98
:1002D0000003040B0C13141A1B24252B2C33343B62
:1002E0003C02050A0D1215191C23262A2D32353A17
:1002F0003D0106090E1116181D2227292E31363907
:100300003E0007080F10171F1E2120282F303738F6
:100310003F0000000000000000000000000000009E
:1003200000000000000000000000000000010101CA
:1003300001010101010101010101020202020202A7
:100340000202030303030303030404040404050576
:10035000050506060606070707070808080909092C
:100360000A0A0A0B0B0B0C0C0D0D0D0E0E0F0F10C5
:10037000101111121213131414151516161718183C
:1003800019191A1B1B1C1D1D1E1F2020212223238F
:10039000242526272728292A2B2C2D2E2F303132B1
:1003A000323334363738393A3B3C3D3E3F404243A6
:1003B00044454648494A4B4D4E4F51525355565766
:1003C000595A5C5D5F606263656668696B6D6E70EB
:1003D00072737577787A7C7E7F81838587898A8C32
:1003E0008E90929496989A9C9EA0A2A4A7A9ABAD39
:1003F000AFB1B4B6B8BABDBFC1C4C6C8CBCDD0D2F8
:10040000D5D7DADCDFE1E4E7E9ECEFF1F4F7F9FC6A
:10041000FF05010906A101050719E029E7150025D7
:100420000175019508810295017508810195057591
:10043000010508190129059102950175039101959E
:10044000067508150026FF000507190029FF810021
:10045000C0050C0901A1018504150026FF03190040
:100460002AFF03950475108100C005010906A1014A
:100470008508050719E029E715002501750195088C
:1004800081020508190129089508750191020507DF
:10049000750495018101190429DD150025017501F7
:1004A00095DA8102750295018101C005010980A1DB
:1004B000018505150026FF00190029FF9501750823
:1004C0008100C0656570726F6D2E65726173650025
:1004D000656570726F6D2E66726565006565707218
:1004E0006F6D2E636F6E74656E7473002F0073658D
:1004F0007474696E67732E637263007365747469D4
:100500006E67732E76657273696F6E0073657474AF
:10051000696E67732E76616C69643F0073657474ED
:10052000696E67732E64656661756C744C6179657C
:1005300072006B65796D61702E6F6E6C79437573A7
:10054000746F6D006B65796D61702E6465666175A1
:100550006C74006B65796D61702E637573746F6D6B
:1005600000454550524F4D4B65796D61700068658F
:100570006C700066616C7365007472756500706CF8
:100580007567696E73006465766963652E7265735D
:1005900065740068656C70000D0A2E004D6F7573F0
:1005A000654B657973004D6163726F73001E08348B
:1005B00008200821082208240834002608270825D6
:1005C000082E0836002D0037003800270033083386
:1005D0000036082E00370838081F082F0031003079
:1005E0000023082D0835002F083108300835086D24
:1005F0006163726F732E74726967676572006D61F3
:1006000063726F732E6D61700044796E616D696302
:100610004D6163726F730070616C65747465006323
:100620006F6C6F726D61702E6D617000436F6C6FD7
:10063000726D6170456666656374004D61676963DC
:10064000436F6D626F0051756B65797300080B0025
:100650000202020000090400000102020000052459
:1006600000100105240101010424020605240600EE
:10067000010705810310004009040100020A00007F
:100680000007050202400000070583024000001237
:10069000010002EF020140091201230001010203DF
:1006A000014B6579626F617264696F004D6F6465BB
:1006B0006C203031000403090405010902A101097D
:1006C00001A10085010509190129081500250195D9
:1006D00008750181020501093009310938158125A4
:1006E0007F750895038106050C0A38021581257F60
:1006F000750895018106C0C005010902A101090123
:10070000A1000509190129081500250195087501A1
:10071000810205010930093116000026FF7F75109E
:100720009502810209381581257F7508950181069A
:10073000C0C0F706F70C090D460D550F271212130E
:100740007013FC1538180D1B0E29682A72313535C7
:10075000FF3511241FBECFEFDAE0DEBFCDBF11E0C1
:10076000A0E0B1E0ECE9FDE602C005900D92AA3FE1
:10077000B107D9F726E0AAEFB1E001C01D92A93474
:10078000B207E1F713E0C9EAD3E004C02197FE0104
:100790000E943A36C939D107C9F70E94D4030C9494
:1007A000CC360C94000008950E94A6040E94D30346
:1007B00082E595E00E9437310E94C406C0E0D0E097
:1007C0000E94F1062097E1F30E940000F9CF1F92EA
:1007D0000F920FB60F9211242F933F938F939F93F5
:1007E000AF93BF938091FB019091FC01A091FD011B
:1007F000B091FE013091FA0123E0230F2D3758F517
:100800000196A11DB11D2093FA018093FB019093E5
:10081000FC01A093FD01B093FE018091FF01909136
:100820000002A0910102B09102020196A11DB11D2A
:100830008093FF0190930002A0930102B093020203
:10084000BF91AF919F918F913F912F910F900FBECC
:100850000F901F90189526E8230F0296A11DB11D39
:10086000D2CF2FB7F8946091FB017091FC01809179
:10087000FD019091FE012FBF08953FB7F89480913C
:10088000FF0190910002A0910102B091020226B5F1
:10089000A89B05C02F3F19F00196A11DB11D3FBFB8
:1008A000BA2FA92F982F8827BC01CD01620F711D87
:1008B000811D911D42E0660F771F881F991F4A9581
:1008C000D1F708958F929F92AF92BF92CF92DF920D
:1008D000EF92FF926B017C010E943D044B015C0191
:1008E000C114D104E104F104E9F00E9471310E94C5
:1008F0003D04681979098A099B09683E734081059E
:10090000910570F321E0C21AD108E108F10888EEE0
:10091000880E83E0981EA11CB11CC114D104E1040F
:10092000F10429F7FF90EF90DF90CF90BF90AF9048
:100930009F908F9008958230910538F0880F991F0D
:10094000880F991F05970197F1F70895789484B55A
:10095000826084BD84B5816084BD85B5826085BDBB
:1009600085B5816085BDEEE6F0E0808181608083A1
:10097000E1E8F0E010828081826080838081816084
:100980008083E0E8F0E0808181608083E1E9F0E04D
:10099000808182608083808181608083E0E9F0E0F3
:1009A000808181608083E1ECF0E0808184608083DD
:1009B000808182608083808181608083E3ECF0E0CD
:1009C000808181608083E0ECF0E0808182608083C0
:1009D000E2ECF0E0808181608083EAE7F0E08081F2
:1009E0008460808380818260808380818160808355
:1009F0008081806880830895FC01892B69F084EAF6
:100A000091E091838083738362831582148281E0F5
:100A1000868317828FEF8087CF010895FC01892B91
:100A200069F080EB91E09183808373836283158208
:100A3000148281E0868317828FEF8087CF0108952B
:100A4000FC01892B79F088E991E09183808373839D
:100A50006283148281E08583809123029091240235
:100A600097838683CF010895009739F020E831E01D
:100A7000FC0131832083738362830895009741F0E2
:100A80002CE831E0FC01318320837383628314827C
:100A90000895009739F02CEB31E0FC01318320837D
:100AA00073836283FB01408308950C942D2584EFAA
:100AB00094E00C943B29089586E0E4E5F1E0DB0145
:100AC00001900D928A95E1F786E00895CF93DF9328
:100AD000EB01882339F08130B9F090E080E0DF91BC
:100AE000CF910895898181FFF8CF80FDF6CF6BE12A
:100AF00071E087E594E00E94171C62EF70E087E5E3
:100B000094E00E94171CE9CF898181FFE6CF80FD28
:100B1000E4CF0E94310424E230E040E050E00E9443
:100B200018366C5F6A831B82D8CF8230910518F02B
:100B3000029719F008950C94AF0C0C94940C0C943B
:100B4000950587E294E00E947F168EEB94E00E9468
:100B5000D32587E594E00E946E1C88E694E00E940D
:100B6000161F8BE091E00E94C6188DE291E00E9472
:100B700054258CE291E00E94032480E008958DE1E9
:100B800094E00E94A11387E294E00E9475168BE026
:100B900091E00E94DA1880EB94E00E94912081E8B5
:100BA00092E00E949F0C8DEA94E00E94DB1F80E09F
:100BB00008958DE194E00E94A0148CEB94E00E94D3
:100BC000372580E00895BC018EEB94E00C946528F5
:100BD000CF93DF93EC01BC0187E594E00E94361CC3
:100BE000811115C0BE0188E694E00E94F31E8111B8
:100BF0000EC0BE018BE091E00E942419811107C054
:100C0000BE0181E892E0DF91CF910C94B90CDF91A5
:100C1000CF910895BC018BE091E00C94DC18CF9348
:100C2000DF93EC01BC0187E294E00E94111781116F
:100C300054C0BE018CE294E00E94E21781114DC0C5
:100C4000BE018CE194E00E94A814811146C0BE014F
:100C50008BE194E00E944B1581113FC0BE018CE2F4
:100C600094E00E94D7178823F9F069EC72E085EFD1
:100C700094E00E94972B84E690E00E949B04BE01C2
:100C800088E694E00E94261F811127C0BE0184EBF4
:100C900094E00E94D222811120C0BE018CE291E03A
:100CA000DF91CF910C94252449EC52E0BE018CE2F7
:100CB00094E00E942E18882311F36FEB72E085EF09
:100CC00094E00E94682B84E690E00E949B0460E21E
:100CD00085EF94E00E948C2BCECFDF91CF910895C9
:100CE0008CE291E00E94172480E0089580E008954E
:100CF00080E00895CF93DF93EC01BC0188E594E098
:100D00000E944B1D811107C0BE0188E594E0DF9170
:100D1000CF910C944B1DDF91CF910895BC018BE0D6
:100D200091E00E94181A80E008958CE294E00E94FD
:100D300072188EEB94E00E94D0288BE091E00E9424
:100D4000F3198DE291E00E94682580EB94E00E9407
:100D5000952081E892E00E94D70B8DEA94E00E94F2
:100D6000472080E00895ECEAF0E0849108959B012B
:100D700094E0899FB001112463557F4F44E050E017
:100D8000C9010C947C36089580915C0190915D01BD
:100D90000E94DC0781E08093AF0466E98AE291E07B
:100DA0000E94C52166E988E291E00E94C82187E39C
:100DB0000E94632487E892E00E94100D85E00E9463
:100DC0009E1665E08CE291E00E94F32360E870E0FB
:100DD00088E694E00E94C21F809121048F770C94D2
:100DE000A20A80915C0190915D010C94FA07EEE1FA
:100DF000F2E020EA208311821282EBE1F2E08CE83B
:100E0000808396E491831282E8E1F2E082E88083B5
:100E100034E631831282E5E1F2E01082218312820E
:100E2000E2E1F2E0108291838283EFE0F2E010824F
:100E300011829AEA9283ECE0F2E08083118288E7E3
:100E4000828308950E94B3110C94FA100E94220725
:100E5000811104C00E94B3110C949B1184EC93E0A7
:100E60000E940C1386EA93E00C94F5110E9422076D
:100E7000811104C00E94B3110C94001184EC93E022
:100E80000E94581286EA93E00C940812CF93C82F60
:100E90000E942207811106C00E94B3116C2FCF91CE
:100EA0000C943C116C2F84EC93E0CF910C94BC1209
:100EB000CF93C82F0E942207811106C00E94B31150
:100EC0006C2FCF910C9463116C2F84EC93E0CF9135
:100ED0000C94E312CF93C82F83FF03C081EE0E94CE
:100EE0004607C0FF03C080EE0E944607C1FF03C053
:100EF00082EE0E944607C2FF03C086EE0E944607AC
:100F0000C4FF04C083EECF910C944607CF9108959F
:100F1000CF93C82F892F0E946A078C2FCF910C94F2
:100F20004607FC019081DB018C91981305C081E09C
:100F3000218111969C91291380E008951F93CF93EE
:100F4000DF9300D000D0CDB7DEB7182F803468F51E
:100F5000E82FF0E0EE0FFF1FE35AFA4F80819181F6
:100F60009C838B838FEF89838A83BE016F5F7F4F62
:100F7000CE0103960E949107882369F0A12FB0E06B
:100F8000A85DBD4FE0910201F0910301612F8C91AA
:100F900009958B839C838B819C810F900F900F9080
:100FA0000F90DF91CF911F9108951092DD0510925F
:100FB000DE05EDEDF5E0D2CF8BE892E00E94460F22
:100FC00040E855E260E070E085EF94E00E94622A1C
:100FD0000E945B050E94BF05EDE5F5E081E49FEF0F
:100FE000815021F0908391833296FACF87E292E08C
:100FF0000C94A00A0E94310460932302709324028F
:10100000809325029093260280912102E09195021F
:10101000F09196020190F081E02D882389F085E916
:1010200092E00995811106C0109221020E94B3112D
:101030000E94AF110E94D9050E94DC0E0C94950607
:1010400085E992E009958823A9F381E08093210244
:10105000F1CFCF93DF93EB01CB010E940A068230E0
:1010600019F1D63419F4C770C052D0E08D2F807CAE
:1010700051F480E28C0F883008F0D0E0CE01DF918F
:10108000CF910C9488078D2F887C883469F46D2F5C
:1010900070E0762F66276C0F711D737086EA93E0FF
:1010A000DF91CF910C94E011DF91CF9108958F9251
:1010B0009F92BF92CF92DF92EF92FF920F931F9376
:1010C000CF93DF9300D000D000D0CDB7DEB77C0146
:1010D0006B010E94260710E000E0BB24BA940034A4
:1010E000110599F1F6019081901729F1003430F53E
:1010F000F801EE0FFF1FE35AFA4F808091809E8225
:101100008D82BB82BC82BE016D5F7F4FCE01059692
:101110000E94910781110FC019821A82BE016F5F70
:101120007F4FCE0105960E949107811104C0B40142
:10113000C7010E9429080F5F1F4FD1CF1092DD0514
:101140001092DE05EDEDF5E0D8CF26960FB6F894B7
:10115000DEBF0FBECDBFDF91CF911F910F91FF90EA
:10116000EF90DF90CF90BF909F908F900895EF9277
:10117000FF920F931F93CF93DF938C01EB01898133
:1011800081FF42C080FD40C08B81807CE9F5888171
:1011900080930101FA800E94220781112FC00E94D2
:1011A000B3116F2D0E94A211882301F1FB80EA8008
:1011B000F3FE03C081EE0E945807F0FE03C080EEEC
:1011C0000E945807F1FE03C082EE0E945807F2FE0B
:1011D00003C086EE0E945807F4FE03C083EE0E940F
:1011E00058078E2D0E9458070E9436078B8188234E
:1011F00081F00E946A070E9436070BC06F2D84ECB5
:1012000093E00E94A612D0CFE09101018881E813FB
:1012100017C0898181FF07C080FD05C06A817B817D
:10122000C8010E942908CE010E947A068230E9F0A6
:10123000DF91CF911F910F91FF90EF900C943607A3
:10124000E03460F4F0E0EE0FFF1FE35AFA4F8181C3
:10125000982F907CF1F60E946A07DBCF1092DD0593
:101260001092DE05EDEDF5E0F2CFDF91CF911F9109
:101270000F91FF90EF900895FF920F931F93CF93DC
:10128000DF93CDB7DEB72D970FB6F894DEBF0FBE54
:10129000CDBF8C0129873A874B875C876D872034C7
:1012A00048F430FF75C031FD73C089850E949E07E8
:1012B0009C878B87CE0109960E94E805823009F44D
:1012C0005BC0E985E03468F49A85F0E0EE0FFF1F1B
:1012D000E35AFA4F90FF69C091FD67C09FEF90837A
:1012E0009183811149C01F821886BE01695F7F4FBB
:1012F000CE010B960E94910781113EC01D821E8275
:10130000BE016B5F7F4FCE010B960E94910781114A
:1013100033C0FF24FA94FB82FC82BE016D5F7F4FD5
:10132000CE010B960E949107811126C0F982FA82A4
:10133000BE016F5F7F4FCE010B960E949107811116
:101340001BC08C858D7F843421F4CE0109960E94C8
:101350002B0B8C85843481F08F7C813499F58A85C0
:101360001B8581FF26C080FD24C0612F8CE094E0A6
:101370000E945813109390022D960FB6F894DEBF7A
:101380000FBECDBFDF91CF911F910F91FF900895B8
:101390008FEF89838A83BE016F5F7F4FCE010B96EB
:1013A0000E949107811181CF85CF9C852B85208359
:1013B00097CF809190028113DFCF8CE094E00E9460
:1013C0005613DACFBE01675F7F4FC8010E945708EE
:1013D000BE01675F7F4FC8010E94B708CE01099622
:1013E0000E948E06C9CFEF92FF920F931F93CF9367
:1013F000DF9300D000D000D01F92CDB7DEB7022F10
:101400002B833C834D835E836F83203408F042C07E
:101410007C01832F817031FF22C081113BC08FEF8F
:1014200089838A83BE016F5F7F4FCE0105960E943C
:101430009107882329F0802F0E949E079E838D8329
:10144000CE0103960E94E305811124C02B813C81CB
:101450004D815E816F81C7010E943C091BC08823BA
:10146000C9F010E0000F111F035A1A4FF8018081D4
:1014700091819E838D8319821A82BE016F5F7F4F97
:10148000CE0105960E9491078823D1F28FEFF801D3
:101490008083818327960FB6F894DEBF0FBECDBF41
:1014A000DF91CF911F910F91FF90EF90089520E46D
:1014B000829FC0011124680F792F711D660F771F5D
:1014C000FB01E15CFE4F8491FB01E05CFE4F9491D7
:1014D0000895EF92FF920F931F93CF93DF93E8E26B
:1014E000F2E080E4DF011D928A95E9F77F0100E0D8
:1014F0000034F9F0C0910401D0E0C859DD4FB2E0EA
:10150000C836DB0789F01A911A3208F01A52E091B6
:101510000201F0910301602F812F09958F3F11F493
:101520009F3F69F3F70110830F5FFFEFEF1AFF0A88
:10153000DFCFDF91CF911F910F91FF90EF90089532
:101540000C94690A90910001891748F491E09093F6
:101550000401809368020E94690A0C947006089541
:10156000CF93C091040190E0BC016F5F7F4F4C2F7F
:1015700050E0461B570B68597D4F88599D4F0E947C
:10158000A436C150C0930401CF9108954091040145
:1015900050E090E0682F70E0292F092E000C330BEB
:1015A0002417350764F428593D4FF9012081022E94
:1015B000000C330B2617370719F09F5FEDCF9FEF15
:1015C000892F0895CF93C82F0E94C60A87FF0AC0AB
:1015D0008AE28C0F0E94C60A8095881F8827881F80
:1015E000CF91089581E0FCCFCF9396ED980F8A328A
:1015F00008F4982F209100019217C8F4C82F0E9478
:10160000C60A87FF0E94B00AE0910401E03110F0A1
:1016100080E0F8CF81E08E0F80930401F0E0E8597C
:10162000FD4FC0830E94690ACF910C947006CF9140
:1016300008950E94C60A87FD0DC090910401923062
:1016400018F480E00C94A20A0E94B00A0E94690A71
:101650000C94700608950F931F93CF93FC01C281E1
:101660009181292F22708381863479F5C695C6959C
:10167000C695C65D8F0186ED8C0F35EB3C0F323081
:1016800008F060C02223E9F090FD1BC0E091040146
:10169000F0E0E959FD4F90819A3208F09A52823277
:1016A000B1F59F5F80910001981798F1D801EC91F6
:1016B000E03438F4F0E0EE0FFF1FE35AFA4F1082E7
:1016C0001182CF911F910F910895C43558F02223B4
:1016D000C1F390FDF6CF8CEA8C0FCF911F910F9143
:1016E0000C94A20ACA3230F6222359F390FDE9CFB6
:1016F00030910401E8E6F2E020E08FEF321789F143
:1017000091919A320CF0982F2F5F892FF7CF91503B
:10171000C9CFCAE2C90F8C2F0E94F40AD801EC91FC
:10172000E03448F4F0E0EE0FFF1FE35AFA4FC083B5
:1017300084E48183C6CF1092DD051092DE05EDEDC5
:10174000F5E0F5CF8C2F222399F090FD11C00E9477
:10175000C60A87FFB6CF8C2FCF911F910F910C94A3
:10176000F40A082E000C990BC8171906A1F78C2F44
:10177000CF911F910F910C94190B8A3208F08A5265
:1017800008950C94AE0D803438F4E82FF0E0EF5259
:10179000FD4F84910C94AE0D8FEFFCCF809106012C
:1017A000882321F00E9478060C94F50D089580910D
:1017B0000601882361F180912302909124022091F7
:1017C000820230918302821B930B2091050128171E
:1017D000190609F0E0F40E94CE0B809105012091DA
:1017E000820230918302820F932F911D9093830286
:1017F000809382028091840290918502009739F053
:10180000DC01ED91FC910480F581E02D099580E0EB
:10181000089580917802811105C01092800281E0C4
:101820008093780280E892E00895CF92DF92EF9261
:10183000CF936B01E82E0E94090CC0E06E2DA6012B
:101840008C2F0E94C10BCF5FC034C1F7CF91EF90B6
:10185000DF90CF90089560E070E080E00E94150C6A
:101860008091840290918502009739F0DC01ED911E
:10187000FC910280F381E02D0994089590918602F5
:10188000891778F4809307010E94120D90938502C6
:10189000809384028091060181110E942B0C0C948C
:1018A00076060895809107018F5F809307019091DC
:1018B0008602891708F080E00C943E0C80910701A5
:1018C000811102C08091860281508093070180912E
:1018D00007010C943E0CEF92FF921F93CF93DF937E
:1018E00000D000D0CDB7DEB77C0110E08091860239
:1018F000181770F4BE016F5F7F4F812F0E94B706EB
:1019000089819A81E816F90669F4812F0E943E0CBC
:101910000F900F900F900F90DF91CF911F91FF903C
:10192000EF9008951F5FE2CF81E0809306010E944F
:101930002B0C0C94F50D762F642F0C94150C60E095
:1019400070E080E00E94150C0E94C30680910701A0
:101950008F3F19F480E00E943E0C80E0089560E023
:1019600070E080E00E94150C0E94F50D10920601B7
:101970000895FB018381833499F5818181FF2BC018
:1019800080FD29C09281EDE5F5E021E4923078F008
:10199000923009F5809106018823F9F00E94AF0C7E
:1019A0001AC0363419F48370813089F03296215090
:1019B000C9F080813181432F407C99F740E2480F84
:1019C0004830A0F78B7F813E11F033FFEFCF9111AC
:1019D0000BC00E945E0C81E008950E94940CFBCF26
:1019E00080E008959111F5CF0E94520CF4CF0E942F
:1019F000B3068093860208950895089560E070E02C
:101A000080E00C94150C862F40E050E060E00C94D0
:101A1000C30B82E691E09093880280938702089539
:101A20000C946B0C1F93CF93DF9300D000D0CDB7F5
:101A3000DEB79091080198130CC0809189029091B3
:101A40008A020F900F900F900F90DF91CF911F910E
:101A50000895182F80930801BE016F5F7F4F0E9489
:101A6000B706EB81FC8189819A81309731F06981D9
:101A70007A81412F83E092E0099590938A028093C6
:101A80008902DBCF82E595E00C944A31EBE8F2E085
:101A900015828EE691E09387828708950E94B311A4
:101AA0000E94F91084EC93E00E94481286EA93E0C9
:101AB0000E94DF118CE094E00C943313CF93DF93FA
:101AC00000D000D01F92CDB7DEB7262F342F842F41
:101AD000817041FF15C0811115C080915C0561E0E6
:101AE000680F60935C054FEF5FEF82E292E00F902A
:101AF0000F900F900F900F90DF91CF910C94F309FE
:101B00008111EBCF0F900F900F900F900F90DF91FE
:101B1000CF9108956E9A769824982C9808958034E1
:101B200020F060E070E080E00895282F30E08032FF
:101B300058F4F901EE0FFF1FE20FF31FED5EFC4FAB
:101B4000608171818281089520523109F901EE0F7F
:101B5000FF1FE20FF31FE755FD4FF2CF0F931F93C7
:101B6000CF93DF93C82F8A01D62F8032F8F40E94DA
:101B70008F0DD81319C081E0171303C0061301C0DD
:101B800080E090910901892B8093090123E0C29F95
:101B9000F0011124ED5EFC4F00831183D283DF91AD
:101BA000CF911F910F91089581E0EBCF8034B8F76A
:101BB0000E948F0DD81317C081E0171303C00613BE
:101BC00001C080E090910901892B809309012C2F9D
:101BD0002052330BC901F901EE0FFF1FE80FF91F67
:101BE000E755FD4FD9CF81E0EDCF809109018823E2
:101BF00011F183E193E00E94161089EA92E00E94BD
:101C0000161083E193E00E94161089EA92E00E9488
:101C1000161083E193E00E94161089EA92E00E9478
:101C2000161083E193E00E94161089EA92E00E9468
:101C300016101092090108953F9A479A08950FB619
:101C4000F894A8958091600088618093600010925C
:101C500060000FBE64E670E080E090E00E946204E5
:101C60000C941C0E8091A5029091A602A091A7024F
:101C7000B091A80280939D0290939E02A0939F0230
:101C8000B093A0028091A1029091A202A091A30220
:101C9000B091A4028093990290939A02A0939B0220
:101CA000B0939C0283E193E00E94960F882361F039
:101CB00083E193E00E94C90F6093A5027093A6028E
:101CC0008093A7029093A80289EA92E00E94960F5F
:101CD000882361F089EA92E00E94C90F6093A10213
:101CE0007093A2028093A3029093A4020895FF929E
:101CF0000F931F93CF93DF93F42E641302C06623D8
:101D0000E1F08295807F182F120F00E0C62FD0E0FF
:101D1000AE01440F551F42708F2D8170482B31F05A
:101D2000612F601B80E090E00E945E0DF6940F5FD3
:101D3000D595C7956C2F083049F7DF91CF911F914A
:101D40000F91FF900895AF92BF92CF92DF92EF92E2
:101D5000FF920F931F93CF938DE9A82E82E0B82EA8
:101D600095EAC92E92E0D92E29E9E22E22E0F22E40
:101D700001EA12E0C0E0F50141915F01F6016191D5
:101D80006F0127E08C2F0E94770EF70141917F01B0
:101D9000F80161918F012FE08C2F0E94770ECF5FA9
:101DA000C43049F7CF911F910F91FF90EF90DF90D2
:101DB000CF90BF90AF9008950E94320E0C94A30E66
:101DC000CF93C82F682F83E193E00E947B0F6C2F85
:101DD00089EA92E0CF910C947B0F282F2F70829587
:101DE0008F7090E0422F50E0283080F48B559D4F4B
:101DF000FC01808190E027E030E0241B350B02C01D
:101E0000959587952A95E2F7817008958F559D4F96
:101E1000FC01808190E02FE030E0EFCF282F2F7081
:101E200082958F7090E0422F50E0283080F48356E6
:101E30009D4FFC01808190E027E030E0241B350BB2
:101E400002C0959587952A95E2F781700895875687
:101E50009D4FFC01808190E02FE030E0EFCF60915A
:101E6000A5027091A6028091A7029091A8020E94FB
:101E70004036282F6091A1027091A2028091A302A6
:101E80009091A4020E944036820F08950E948A0D0C
:101E90000E944E0D0E941F0E8CE08093B8000895A2
:101EA0005D9A289A82E00C94E00E60E083E193E072
:101EB0000E945F0F63E089EA92E00C945F0FFC01DF
:101EC000E05AFF4F1082399610823697262F30E065
:101ED000318320838F599F4F686570E0FC017183C7
:101EE000608380910A019FEF980F90930A018111FE
:101EF0000C94193208950F93CF93DF9300D0CDB790
:101F0000DEB722E029836A838F599F4F00E021E0EA
:101F100042E0BE016F5F7F4FFC0180810E947932F9
:101F20000F900F90DF91CF910F9108950F931F9312
:101F3000CF93DF9300D000D01F92CDB7DEB78C01D6
:101F4000FC01EF59FF4F21E045E0BE016F5F7F4F7D
:101F500080810E94313289818130C9F4F801EB59C6
:101F6000FF4F8A81808331968B81808331968C816B
:101F7000808331968D81808381E00F900F900F9048
:101F80000F900F90DF91CF911F910F91089580E0F6
:101F9000F4CF8B599F4FFC016081718182819381C5
:101FA00008950F93CF93DF93CDB7DEB769970FB640
:101FB000F894DEBF0FBECDBF20E8260F2983FC01B9
:101FC000E05AFF4F4081DE01129628E1629FB00186
:101FD000112430E020E0F901E60FF71FE80FF91FA8
:101FE000E0814E1708F5E41BF0E0EF5EFC4FE49152
:101FF000ED932F5F3F4F2831310569F78F599F4F80
:1020000000E021E049E1BE016F5F7F4FFC0180816C
:102010000E94793269960FB6F894DEBF0FBECDBF2D
:10202000DF91CF910F910895E0E0DECFCF93DF9362
:10203000EC01C759DF4F688121E0260F28830E94F9
:10204000D10F8881843009F41882DF91CF910895EF
:10205000FC0182818F5BFB01808381E00895CF9337
:10206000DF93CDB7DEB769970FB6F894DEBF0FBE2A
:10207000CDBFFC01DB019C919F5F9C939E012D5F76
:102080003F4F81E1D9011D928A95E9F729E0298323
:1020900084E08A8391E09D8383E08E839F83988789
:1020A0002A8721E22B879C879D879F8722E2288BA6
:1020B00020E4298B27E02B8B25E02C8B8E8B20E4D2
:1020C00030E0388F2F8B998F82818B83838180685A
:1020D0008D8B49E150E0BE016F5F7F4F80E00E9431
:1020E000112F69960FB6F894DEBF0FBECDBFDF91FA
:1020F000CF910895FB012081213891F42381223270
:1021000079F4DC0112962C918481958128171906A7
:1021100039F440E450E061E174E080E80C94112F60
:1021200090E080E00895FC01DB01228114968D91FE
:102130009C9115972817190691F511968C91119776
:102140009C91913A69F4813029F0833029F4848D8F
:102150008093F10081E00895823009F5858DF8CFF4
:102160009132E9F48B3021F412968C91848FF2CF66
:102170008A3021F412968C91858FECCF893079F4D6
:10218000CF0116962D913C91179713964C914230A2
:1021900041F461E070E04E962130310551F080E06D
:1021A00008954130E1F728303105C9F768E070E063
:1021B0000B960E94372FCECFCF93DF93EC0181E0B7
:1021C0008C838D83CE014B969F838E8319861886D0
:1021D00084E791E0998388836A876C8F1D8E1E8EB9
:1021E00081EC8B8F0E94452BBE01DF91CF910C9427
:1021F000012B0895FC01848D0895FC01648F0895DE
:10220000EF92FF920F931F93CF93DF938C01EC011A
:102210002B967C0183E1E80EF11C48E050E0BE0102
:10222000C7010E948E36892B21F1F801838148E095
:1022300050E0BE0180640E94602E8C01E091A403F6
:10224000F091A503309731F09C0148E050E0BE01C9
:1022500082E0099588E0FE01D70101900D928A95F0
:10226000E1F7C801DF91CF911F910F91FF90EF909F
:1022700008950FEF1FEFF5CFFC0180E2860F883045
:1022800070F4605E770B21E030E001C0220F6A95A8
:10229000EAF78385822B838781E090E00895DF0150
:1022A0001D9690E080E02D912617B1F3211104C016
:1022B000E80FF91F6587F0CF01968630910599F7F1
:1022C00090E080E00895CF93DF9320E2260F28303E
:1022D00090F4605E770B21E030E001C0220F6A9538
:1022E000EAF72095FC0133852323238781E090E0E2
:1022F000DF91CF910895DC011D969C012D5E3F4F2B
:10230000FD014191461303C0EF0121971882E217A6
:10231000F307B9F720E03D91332349F0EC01C20FF8
:10232000D11D4D853D87ED01219748832F5FAE1765
:10233000BF0789F7DBCF0B9628E0FC0111922A95A5
:10234000E9F70895FC013D9643962191261729F05F
:10235000E817F907D1F780E0089581E00895FC01BE
:102360002285248F089580917D03811108C061E04A
:1023700085E893E00E94DC1081E080937D0385E88E
:1023800093E008958091B603811113C01092BF03AA
:102390001092BE0381E594E09093C1038093C00343
:1023A00089E190E09093C3038093C20381E080931E
:1023B000B6030E94CD346EEB73E00C94383408956C
:1023C000FC0130E020E041915191452B41F4220F76
:1023D000331F280F391FF9017183608308952F5F20
:1023E0003F4F2430310579F7089528E0FC01119220
:1023F0002A95E9F70895CF93DF93EC010E94CD343D
:1024000028E030E0AE0164E0DF91CF910C94883495
:102410000F931F93CF93DF93EC018C01085F1F4F45
:1024200048E050E0BC01C8010E948E36892B51F073
:10243000CE010E94FB1188E0FE01D80101900D92AF
:102440008A95E1F7DF91CF911F910F91089586EA68
:1024500093E00C94C2118091FE03811113C010927D
:102460000704109206048AE694E09093090480938E
:10247000080481E490E090930B0480930A0481E0C7
:102480008093FE030E94CD3466E074E00C943834EF
:102490000895CF93DF93EC010E94CD34AE01435EEB
:1024A0005F4F2DE130E068E0DF91CF910C948834EC
:1024B000EF92FF920F931F93CF93DF93EC01F8807D
:1024C0008D8D8E010F5F1F4F8F15D9F0F801AE0172
:1024D000435E5F4F20E0858D30813196932F90953C
:1024E000982319F08323848F21E0E417F50799F7E7
:1024F000222319F0CE010E944912FD8ECE010E94C6
:1025000049127E018EE1E80EF11C4CE150E0B80169
:10251000C7010E948E36892B81F08CE1F801D7012A
:1025200001900D928A95E1F7CE01DF91CF911F9135
:102530000F91FF90EF900C9449128FEF9FEFDF9176
:10254000CF911F910F91FF90EF9008956E3D90F401
:10255000E62FE695E695E695E80FF92FF11D6770F1
:1025600021E030E001C0220F6A95EAF791819223C1
:1025700081E009F480E008956E3DA0F4E62FE69531
:10258000E695E695E80FF92FF11D677021E030E040
:1025900001C0220F6A95EAF78181822B818381E055
:1025A00090E00895605E683058F441E050E001C06A
:1025B000440F6A95EAF7FC012081242B2083EFCF9A
:1025C00090E080E008956E3DA8F4E62FE695E6954C
:1025D000E695E80FF92FF11D677021E030E001C0AA
:1025E000220F6A95EAF7209581812823218381E0D3
:1025F00090E00895605E683060F421E030E001C052
:10260000220F6A95EAF72095FC013081232320836D
:10261000EECF90E080E008952DE1FC0111922A9523
:10262000E9F7089584EC93E00C942B1280910D044B
:10263000811113C010921604109215048BEA94E0D5
:10264000909318048093170488E190E090931A0403
:102650008093190481E080930D040E94CD3465E1DC
:1026600074E00C94383408950F931F93CF93DF9345
:10267000EB018A010E94CD349801AE0165E0DF9143
:10268000CF911F910F910C948834CF93DF931F92B9
:10269000CDB7DEB7198241E050E0BE016F5F7F4FDA
:1026A0000E9434130F90DF91CF9108950C9445133D
:1026B000CF93DF931F92CDB7DEB76983633841F4C0
:1026C00082E595E00E9451310F90DF91CF910895FE
:1026D00041E050E0BE016F5F7F4F0E943413F4CFA2
:1026E0008CE094E00C94161384E690E00C949B0428
:1026F0004AE050E0682F85EF94E00E94512C0E9440
:10270000741360E285EF94E00E948C2B0C94741398
:10271000FF920F931F93CF93DF93EC01F62E088166
:102720001981C8010E94B636F81621F06F2DC80134
:102730000E94BE36CE01DF91CF911F910F91FF9085
:102740000895AF92BF92CF92DF92EF92FF920F93D4
:102750001F93CF93DF9300D0CDB7DEB78C016C0110
:1027600084E0C80ED11C5601F12CE12CC7010E9457
:10277000B636F50181935F01FFEFEF1AFF0A84E09F
:10278000E816F10499F7F80185818F3FD1F484812F
:10279000982F9F779F3711F487FD148281E0F8010D
:1027A000858310E000E01A830983F60161916F01CF
:1027B000CE0101960E9488130F5F1F4F0430110550
:1027C00091F780E00F900F90DF91CF911F910F91C3
:1027D000FF90EF90DF90CF90BF90AF9008950F9350
:1027E0001F93CF93DF9300D0CDB7DEB77A83698391
:1027F000FC01238110E000E021110FC00081118154
:10280000CB01800F911F9183808342E0BE016F5FF7
:102810007F4F85E294E00E941C16C8010F900F9034
:10282000DF91CF911F910F910895CF92DF92EF9298
:10283000FF920F931F93CF93DF9300D0CDB7DEB7F6
:102840007C016C0184E0C80ED11C10E000E01A830A
:102850000983F60161916F01CE0101960E948813F0
:102860000F5F1F4F0430110591F781E0F70182835C
:102870000F900F90DF91CF911F910F91FF90EF90EC
:10288000DF90CF9008951F93CF93DF93EC01162F25
:1028900080910001681748F4862F0E94A20A8C815B
:1028A0008078912F9F77892B8C831E3720F08C8125
:1028B00080788E678C83CE010E9415148C818F776F
:1028C000DF91CF911F910895FC01948160FB97F9EE
:1028D0009483892F8F778F3719F490789E6794832C
:1028E000CF010C941514CF93DF93EC0181E08B831F
:1028F00060E185E294E00E9403168D81813021F031
:102900001A82DF91CF9108952E813F818091250415
:10291000909126042F3F320779F49F838E83CE0156
:102920000E94151481E08A838C818F778E3748F757
:10293000DF91CF910C94A20A2817390711F7F2CF33
:10294000FC012381211102C00E94731480E00895CC
:10295000CF93DF93EB018CE294E00E94D71788239A
:1029600011F16CE175E085EF94E00E94972B0E94D5
:1029700074136CE075E085EF94E00E94972B0E9441
:1029800074136BEF74E085EF94E00E94972B0E9424
:1029900074136EEE74E085EF94E00E94972B0E9412
:1029A000741380E061C04CE155E0BE018CE294E01C
:1029B0000E942E18882391F08CE294E00E943B182C
:1029C000811165C041E070E060E085EF94E00E9415
:1029D000C62C8DE194E00E94431445C04CE055E0C4
:1029E000BE018CE294E00E942E18811140C04BEF92
:1029F00054E0BE018CE294E00E942E1881112FC099
:102A00004EEE54E0BE018CE294E00E942E18882322
:102A100041F280912004D0E0C0E0882321F0C091F1
:102A20002304D091240460912504709126044AE087
:102A300050E085EF94E00E94582C0E9474136CEED5
:102A400074E085EF94E00E94682B0E9474134AE0C2
:102A500050E0BE0185EF94E00E94582C15C0809193
:102A600022040E94781381E0DF91CF910895609154
:102A70001F048CE294E00E94CC170E94741360E261
:102A800085EF94E00E948C2B0E947413ECCF809110
:102A900021048F77E6CF0F931F93CF93DF9300D05E
:102AA000CDB7DEB78B018CE294E00E94D717882364
:102AB00001F16CED74E085EF94E00E94972B0E9489
:102AC000741360ED74E085EF94E00E94972B0E94F0
:102AD000741363EC74E085EF94E00E94972B0E94DE
:102AE000741380E00F900F90DF91CF911F910F91A1
:102AF00008954CED54E0B8018CE294E00E942E1849
:102B0000882311F18CE294E00E943B1810E000E071
:102B1000811166C08CE294E00E943B1881115EC076
:102B200041E070E060E085EF94E00E94C62C1A83DB
:102B30000983CE0101960E9488130F5F1F4F011574
:102B400084E0180739F74AC040ED54E0B8018CE240
:102B500094E00E942E1881112AC043EC54E0B80181
:102B60008CE294E00E942E18882309F4BBCF10E079
:102B700000E01A8309836FEFCE0101960E9488134B
:102B80000F5F1F4F011584E0180799F787E797E754
:102B9000909301088093000888E19BE00FB6F894B9
:102BA000A895809360000FBE90936000FFCF809146
:102BB0001D0490911E0460E074E0681B790B4AE0EC
:102BC00050E085EF94E00E94582C0E94741360E25C
:102BD00085EF94E00E948C2B0E94741381E082CFD9
:102BE000C8010E94B6360E9478130F5F1F4F01156F
:102BF00084E01807A9F7F2CF84E090E090931E04D8
:102C000080931D040895FC012081318121703327B8
:102C100081E0861770F44081518156954795518324
:102C20004083220F331F41705527242B352B8F5F94
:102C3000F0CF318320830895DC01FB01415000F186
:102C400081912D913C91119768E070E051E0982FAF
:102C5000952399F4932F991F9927991F220F331FBA
:102C6000992319F095E029273058550F61507109C3
:102C700071F711963C932E93E1CF932F9095EBCF64
:102C8000089584E690E00C949B041F93CF93DF9308
:102C900090912904891730F080E090E0DF91CF9186
:102CA0001F910895C62F20E4829FC0011124C80FF0
:102CB000D92FD11DCC0FDD1F60912A0470912B04F8
:102CC000C60FD71FCE010E94B636182FCE0101962F
:102CD0000E94B636912FE2CF90912804891710F404
:102CE0000C94570A891B0C9445168DE194E00E94C0
:102CF000A113809100018093280480E0089561E68B
:102D000075E085EF94E00E94682B0E94411685EFE4
:102D100094E00E94932B0E94411680E008958093D6
:102D2000290490E8899FB00111248DE194E00E946C
:102D3000EF1390932B0480932A040895809300014D
:102D40009091210425E436E197FD07C09091280475
:102D5000980F909300012CE636E130930301209305
:102D600002010C948F16FF920F931F93CF93DF9362
:102D700000D0CDB7DEB7F62E672F8C01000F111FE4
:102D800080912A0490912B04800F911F9A8389834C
:102D9000CE0101960E94881380912A0490912B0401
:102DA0000196800F911F9A8389836F2DCE01019622
:102DB0000E9488130F900F90DF91CF911F910F9178
:102DC000FF900895FF920F931F93CF93DF93F82EF8
:102DD0008B01C0E0CF15F9F0D0E06D2F8C2FF801FA
:102DE0000995692F70E0762F6627680F711D4AE0FC
:102DF00050E085EF94E00E94582C0E94411660E25A
:102E000085EF94E00E948C2B0E944116DF5FD03446
:102E100021F7CF5FDFCFDF91CF911F910F91FF900F
:102E200008950F931F93CF93DF931F92CDB7DEB713
:102E30008B018CE294E00E94D7178823F9F063E5B8
:102E400075E085EF94E00E94972B0E94411664E4A0
:102E500075E085EF94E00E94972B0E94411662E393
:102E600075E085EF94E00E94972B0E94411680E068
:102E70000F90DF91CF911F910F91089542E355E09C
:102E8000B8018CE294E00E942E188823F1F18CE2C4
:102E900094E00E943B188823B1F06091210467FB05
:102EA000662760F94AE050E085EF94E00E94512CDB
:102EB0000E94411660E285EF94E00E948C2B0E94F4
:102EC000411681E0D5CF41E070E060E085EF94E00D
:102ED0000E94C62C162F69838DE194E00E94641431
:102EE0009091290490930001112339F085E496E133
:102EF0009093030180930201E4CF80912804890F0D
:102F0000809300018CE696E1F3CF44E455E0B801EC
:102F10008CE294E00E942E18882339F067E57AE06D
:102F2000809128040E94E216CCCF43E555E0B80119
:102F30008CE294E00E942E18882309F498CF8CE24A
:102F400094E00E943B1810E000E0882329F065E43B
:102F500076E180912904E6CF8CE294E00E943B1850
:102F60008111AFCF8091290420E4829FC0011124F8
:102F70000817190708F0A5CF41E070E060E085EF81
:102F800094E00E94C62C272F3327722FC8010E947D
:102F9000B3160F5F1F4FE0CF611106C063E775E006
:102FA00085EF94E00C94682B69E775E0F9CFCB01CD
:102FB0006EE675E00E94853621E0892B09F020E05D
:102FC000822F0895CF93DF93EB010E94D7178823B8
:102FD00001F163E975E085EF94E00E94972B84E6A8
:102FE00090E00E949B0466E875E085EF94E00E9403
:102FF000972B84E690E00E949B046EE775E085EFD6
:1030000094E00E94972B84E690E00E949B0480E06D
:1030100022C066E875E0CE010E948536892B89F4CE
:1030200087E797E7909301088093000888E19BE089
:103030000FB6F894A895809360000FBE909360003F
:10304000FFCF6EE775E0CE010E948536892BF9F639
:103050000E94A10581E0DF91CF910895CB01BA01D3
:103060000E94853621E0892B09F020E0822F089507
:1030700010924C0408958F929F92AF92BF92CF927C
:10308000DF92EF92FF92C090F904D090FA04E090A2
:10309000FB04F090FC040E9431044B015C0185EFBD
:1030A00094E00E947429082E000C990B8A30910537
:1030B00069F097FF15C00E943104681979098A09DF
:1030C0009B096C157D058E059F0548F381E0FF90F7
:1030D000EF90DF90CF90BF90AF909F908F9008952A
:1030E00080E0F5CFCF93DF93EC0185EF94E00E9471
:1030F0008A2985EF94E00E948D29892B09F442C02A
:1031000085EF94E00E9474298A3099F185EF94E06C
:103110000E949D2980329105E1F4CE010E940F06A4
:1031200085EF94E00E948D29892B31F085EF94E0A2
:103130000E949D290A97A1F768E975E085EF94E060
:103140000E94972B18A280E2FE0111928A95E9F75E
:1031500019C0E8A191E09E0F98A3EC0FFD2FF11D7F
:1031600080839F3130F485EF94E00E948D29892B74
:1031700039F685EF94E00E9474290A9771F288A1CC
:103180008F3158F680E0DF91CF9108956CE975E0BA
:1031900085EF94E00E94682B84E690E00E949B04F7
:1031A00085EF94E00E94932B84E690E00E949B04BC
:1031B00080E0089580E00895FC01703579F4862F51
:1031C0008076803429F49485862F8F7B892B8487A1
:1031D000862F807729F48385682B638780E00895A4
:1031E0008031E1F780E1689FB0011124F4CFCF93E3
:1031F000DF93EC0181E296E00E9402356C8581E26A
:1032000096E00E94083581E296E0DF91CF910C9420
:103210001A35FB01828186FB992790F960E080FDD9
:1032200062E0692B90E081FD94E0692B90E082FDE3
:1032300098E0692B83FD06C080E0682B8EE494E063
:103240000C949B1A80E1F9CFFB0123812035A9F46E
:10325000DC011B961C921B9722812076203411F4EE
:103260001C961C92218121FF08C020FD06C0BF01D1
:10327000228125FF04C00E94091980E008958EE490
:1032800094E00E94981AF9CF609123027091240271
:10329000FC0126813781621B730B23813481261741
:1032A000370760F090E080E0982F872F762F662711
:1032B00050E040E00E941836822F08958FEF089565
:1032C000482F50E087FD0AC0889FC0011124880F55
:1032D000892F881F990B91958F5F089520E031E029
:1032E000241B350B229FC001239F900D900D1124AC
:1032F000880F892F881F990B919580950895CF93FA
:10330000DF93EC010E9444190E94601929819A817F
:10331000921B30E0322F2227989F200D311D11245F
:1033200054E0369527955A95E1F7220F331F220F67
:10333000331F80914D0490E0805C9F4F280F391F10
:1033400020934D04832FDF91CF9108950F93CF9356
:10335000FC01C2852C2F2F70D1F00E947F19682F9D
:103360006195C2FF60E0C3FD680F482F4195C0FF23
:1033700040E0C1FD480F00E020E081E296E00E94BD
:10338000FA3481E296E0CF910F910C941A35CF91E7
:103390000F9108950F93FC01828590E054E095957C
:1033A00087955A95E1F70097E1F09C0136952795AE
:1033B000369527952170022F019583FF02C001E009
:1033C000021B9C012170332781FD215040E060E009
:1033D00081E296E00E94FA3481E296E00F910C942B
:1033E0001A350F910895CF93DF93FC012285222394
:1033F000D9F0EC01809123029085891B843030F054
:10340000CF010E94A61988858C5F8887809123024E
:103410009985891B9881891738F0CE010E94CA19B5
:1034200089859881890F898780E0DF91CF91089500
:103430000F931F93CF93DF93FB012381203521F559
:103440008B01EC0182818076803419F4CE010E94D8
:10345000F7188A858F7031F48091230290912402AD
:103460009F838E838B858A871B86F801818181FFEC
:103470000BC080FD09C08281807761F4CE010E947B
:10348000A61980912302888780E0DF91CF911F9158
:103490000F9108958031C1F7CE010E94CA19809121
:1034A00023028987F1CF0F931F93CF93DF9300D02F
:1034B00000D000D0CDB7DEB716950795600F711F0D
:1034C00036952795420F531FE5E3F6E0758764872D
:1034D00057874687808989837B836A835D834C8392
:1034E0001E820284F385E02D0190F081E02D46E0FC
:1034F00050E0BE016F5F7F4F8FE396E009952696FF
:103500000FB6F894DEBF0FBECDBFDF91CF911F91F4
:103510000F910895FC0117821682158214828FEF95
:103520009FE7918380839383828381E080870895DE
:10353000FC0110860895FF920F931F93CF93DF93A2
:10354000EC01F62E8885811103C0CE010E948A1AF3
:10355000F0FE07C01886DF91CF911F910F91FF9069
:1035600008956091100170E0888199810E9404366D
:103570008B01798368836091100170E08A819B815F
:103580000E9404369B017B836A836F2D64704C819B
:103590005D818E819F817F2D7670763069F4B801D0
:1035A000680F791F7F836E83420F531F5D834C83A7
:1035B000CE010E94531ACFCF662329F1E09110016A
:1035C000E150FF0BE29FB001E39F700DF29F700D81
:1035D0001124460F571F5D834C83F4FE19C04091A0
:1035E00010014150550B409FB001419F700D509FFD
:1035F000700D1124860F971F9F838E834C815D81F0
:103600006E817F81D5CFF1FCE8CF420F531FE3CF0E
:10361000F3FCF4CF800F911FEFCF10925604089562
:10362000FC0184913196949108958F929F92AF926C
:10363000BF92FF920F931F93CF93DF93EB012097DD
:1036400009F4A4C0F12C8E010F5F1F4FFE0184917D
:10365000EFEFE80FED3008F099C0F0E0EE5CF44ECB
:103660000C943A366F1B7B1B841B911B9E1BAB1B60
:10367000B41BBD1B731B731B731B3F1B5A1B8F2C6F
:10368000912CB12CA12CB801F80184916F5F7F4F70
:103690000E5F1F4FFB016491611102C0882319F175
:1036A000782F88E594E00E94261DC501B4010E9490
:1036B0006204E9CF8F2C912CB12CA12C0F5F1F4FEE
:1036C000F80131976491662371F070E088E594E029
:1036D0000E94261DC501B4010E946204EFCF22960C
:1036E000F801F4908E016F2D70E090E080E00E9470
:1036F0006204E801A8CF2296F801649170E090E09E
:1037000080E00E946204EECFF80174918E010D5F9B
:103710001F4FFE013296649188E594E00E94821C5E
:10372000E2CFF80174918E010D5F1F4FFE013296BA
:10373000649188E594E00E94BD1CD5CFF801749196
:103740008E010D5F1F4FFE013296649188E594E073
:103750000E94261DC8CF2296F801649170E088E58A
:1037600094E00E94821CBECF2296F801649170E022
:1037700088E594E00E94BD1CB5CF2296F8016491C3
:1037800070E088E594E00E94261DACCFDF91CF91D8
:103790001F910F91FF90BF90AF909F908F900895D1
:1037A000862F90E06134E0F46A33B0F5603269F15D
:1037B00070F46A3039F130F482E2683050F590E00C
:1037C00080E008956B31D9F790E089E20895613384
:1037D000F8F4880F991F85599A4F0E94101B08957D
:1037E000613638F46B35E8F0880F991F8B5D9A4F7E
:1037F000F4CF6B37D0F06F3710F7880F991F8F50C9
:103800009B4FEBCF90E088E2089590E08CE2089522
:103810008DEE860F90E00895880F991F875A9A4F72
:10382000DCCF83EC860F98E0089583EAF2CF0F9304
:103830001F93CF93DF938C01EB01FE01649166230C
:1038400071F0C8010E94D01B811102C0992329F098
:10385000BC0188E594E00E94261D2196EECF90E001
:1038600080E0DF91CF911F910F9108950F931F93E7
:10387000CF93DF93EB012B8130E0322F22274A8157
:1038800050E0BA017056260F371F2F3F310509F05F
:10389000F8F48C01BE01842F0E946605BC01C801AA
:1038A0000E94151B898180FF02C081FF0DC08A81A3
:1038B00090E090562B8130E0322F2227820F931F09
:1038C0008F3F910529F020F088E594E00E94E51CE7
:1038D00080E0DF91CF911F910F91089566EA75E026
:1038E00085EF94E00E94682B84E690E00E949B04A0
:1038F00085EF94E00E94932B84E690E00E949B0465
:1039000080E00895EF92FF920F931F93CF93DF9380
:1039100000D000D01F92CDB7DEB78C01F62EE72E77
:1039200060915C058FEF898382E88A83FB827C83C8
:103930006D832FEF32E84F2D572F82E292E00E94E5
:103940003C09C8014096F801E817F90741F02081C9
:10395000211111C0218121110EC0F082E1820F904E
:103960000F900F900F900F90DF91CF911F910F91BB
:10397000FF90EF9008953296E7CFCF93DF9300D07A
:1039800000D01F92CDB7DEB7AB019C01205F3F4F47
:10399000FC012E173F0751F08081841305C08181FF
:1039A000851302C0108211823296F3CF60915C05BC
:1039B0002FEF31E882E292E00F900F900F900F907E
:1039C0000F90DF91CF910C943C09CF92DF92EF9250
:1039D000FF920F931F93CF93DF9300D000D01F92DD
:1039E000CDB7DEB77C0120E1E20EF11C8C01DD24B5
:1039F000DA9481E8C82EE016F106D1F0F801408192
:103A00005181411102C0552381F060915C05D9823A
:103A1000CA824B835C836D832FEF31E882E292E0B0
:103A20000E943C09F801108211820E5F1F4FE3CF04
:103A30000F900F900F900F900F90DF91CF911F91EB
:103A40000F91FF90EF90DF90CF9008950F931F9309
:103A5000CF93DF9300D000D01F92CDB7DEB78B019C
:103A600060915C052FEF32E8A80182E292E00E94AB
:103A70003C0960915C052FEF31E8A80182E292E0F9
:103A80000F900F900F900F900F90DF91CF911F919B
:103A90000F910C943C090F931F93CF93DF938C01EC
:103AA000005F1F4FEC010C171D0771F068817981D1
:103AB00089819881911102C0882321F082E292E0ED
:103AC0000E9429082296EFCF80E0DF91CF911F91CD
:103AD0000F91089584E690E00C949B040C94B63604
:103AE0008F929F92AF92BF92CF92DF92EF92FF920E
:103AF0000F931F93CF93DF938C01FC01E080F18043
:103B000015821482C280D380CE0CDF1C4701B12CF9
:103B10008C149D0408F04BC0E4012196C4010E945E
:103B20006E1D8E3008F043C0E82FF0E0E656F24EEE
:103B30000C943A36C91DA81DA81DAC1DAC1DAC1DAA
:103B4000A81DA81DA81DAA1DAA1DAA1DAF1DBE1D2A
:103B5000E40122964E01DCCFE4012396FBCF4E0117
:103B6000CE010E946E1DA82E2296C40101960E94CD
:103B70006E1DA110F4CF8111F2CFECCF2C2F9D2F11
:103B80002196822F0E946E1D2C2F9D2F8111F8CF20
:103B9000E1CFB394EB2DF0E03296EE0FFF1FE00F74
:103BA000F11FCE018E199F0991838083D3CF8B2D76
:103BB000DF91CF911F910F91FF90EF90DF90CF9009
:103BC000BF90AF909F908F9008958F929F92AF92E9
:103BD000BF92CF92DF92EF92FF920F931F93CF93FA
:103BE000DF93FC01EC5BFF4F2081621708F0DFC020
:103BF0007C01E62FF0E03296EE0FFF1FEE0DFF1D69
:103C0000D7010D911C9180819181080F191FD12C32
:103C1000F7018081918122813381820F931F0817E0
:103C2000190708F0C4C0E8012196C8010E946E1D62
:103C300081508D3008F0BBC0E82FF0E0EE5DF14E12
:103C40000C943A364E1E5D1E691E7A1E8B1E9C1EFB
:103C5000A81EB41E551E551E551E2F1EC01E8D2C8F
:103C6000912CB12CA12CCE010E946E1DC82E8E016C
:103C70000E5F1F4FCE0101960E946E1D811102C082
:103C8000CC2091F0682F7C2D88E594E00E94261DC1
:103C9000C501B4010E946204E801E5CF0E5F1F4F29
:103CA000CE010E946E1DD82EE8016D2D70E090E0CF
:103CB00080E00E9462048E01ABCF0E5F1F4FCE01E9
:103CC0000E946E1D682F70E090E080E00E94620408
:103CD000EBCFCE010E946E1DC82EE8012396C801CD
:103CE00002960E946E1D682F7C2D88E594E00E944C
:103CF000821CDBCFCE010E946E1DC82EE8012396E8
:103D0000C80102960E946E1D682F7C2D88E594E004
:103D10000E94BD1CCACFCE010E946E1DC82EE801B4
:103D20002396C80102960E946E1D682F7C2D88E59F
:103D300094E00E94261DB9CF0E5F1F4FCE010E9456
:103D40006E1D682F70E088E594E00E94821CACCF65
:103D50000E5F1F4FCE010E946E1D682F70E088E538
:103D600094E00E94BD1CA0CF0E5F1F4FCE010E94A9
:103D70006E1D682F70E088E594E00E94261D94CFA8
:103D8000CE018D2C912CB12CA12C21960E946E1D60
:103D9000882309F48ACF682F70E088E594E00E94B8
:103DA000261DC501B4010E946204CE01EECFDF9151
:103DB000CF911F910F91FF90EF90DF90CF90BF9028
:103DC000AF909F908F900895292F30E0322F2227B7
:103DD00090E08C55914D280F391F81E0203231053C
:103DE00008F080E008950F931F93CF93DF938C0129
:103DF000EB018A819B810E94E41E8823A9F08981BE
:103E000081FF0DC080FD0BC06A816C55C8010E9406
:103E1000E51D81E0DF91CF911F910F91089588E515
:103E200094E00E94E51CF5CF80E0F4CF69E076E0F5
:103E300085EF94E00E94682B0E946A1D85EF94E054
:103E40000E94932B0E946A1D80E00895CF92DF921A
:103E5000FF920F931F93CF93DF93EC018B018CE2C2
:103E600094E00E94D717882391F06EEF75E085EFFC
:103E700094E00E94972B0E946A1D6FEE75E085EF1B
:103E800094E00E94972B0E946A1D80E05EC04EEF76
:103E900055E0B8018CE294E00E942E18882309F4C2
:103EA0005CC08CE294E00E943B1810E000E08823A4
:103EB000F9F08A819B810817190708F045C08881AD
:103EC0009981800F911F0E946E1D4AE050E0682F7B
:103ED00085EF94E00E94512C0E946A1D60E285EFFC
:103EE00094E00E948C2B0E946A1D0F5F1F4FE1CF50
:103EF0008CE294E00E943B18811120C08A819B8152
:103F000008171907D8F441E070E060E085EF94E00D
:103F10000E94C62CF62E68018FEFC81AD80A888135
:103F20009981080F191FC8010E94B636F81621F0B2
:103F30006F2DC8010E94BE368601DACFCE010E94E5
:103F4000701DCC5BDF4F888381E0DF91CF911F91A3
:103F50000F91FF90DF90CF9008954FEE55E0B8019C
:103F60008CE294E00E942E18882309F48ECF41E061
:103F700070E060E085EF94E00E94C62CCE010E94C4
:103F8000E51DE2CF0F931F93CF93DF93EC018B01DD
:103F90008DE194E00E94EF13998388831B830A8349
:103FA000CE010E94701DCC5BDF4F8883DF91CF91E3
:103FB0001F910F91089580E00895EF92FF921F9353
:103FC000CF93DF93809107010E943E0C88E2E82E98
:103FD00082E0F82EC0E0E0910201F09103016C2F25
:103FE000D7018D917D010995182FD92FE0910201FC
:103FF000F09103016C2F8091AF0409952091AF04DB
:10400000211304C0D43411F4C09318011817F1F02F
:104010008091840290918502009751F5CF5FC03462
:10402000D1F680911801803460F540E06FEF809107
:1040300019010E94E931AB01682F80911801DF91CD
:10404000CF911F91FF90EF900C94C30BD913E0CF49
:10405000111102C0DD23E1F2D111DACF40911A0132
:1040600050911B0160911C018C2F0E94C30BD6CF75
:10407000DC01ED91FC910680F781E02D6C2F099514
:10408000CDCFDF91CF911F91FF90EF900895CF9307
:10409000DF93EC018091AF040E94E20A9091AE049C
:1040A00081110CC0992331F0809107010E943E0CD0
:1040B0001092AE0480E0DF91CF910895911103C07A
:1040C00081E08093AE04CE010E94DD1FF3CF0F93F9
:1040D0001F93CF938091220108E212E0C0E0803468
:1040E00048F48093230181E08093B30416C0CF5F2E
:1040F000C034C9F3E0910201F09103016C2FD801A3
:104100008D918D010995209120012813F0CF809188
:1041100021018913ECCFC0932301CF911F910F91FF
:1041200008950E94672080E008958091B304811172
:1041300023C080912302909124022091B1043091F8
:10414000B204821B930B20911D0130911E01821736
:104150009307A0F081E08093B304609123018091E4
:10416000840290918502009739F0DC01ED91FC9179
:104170000680F781E02D099580E0089540E06FEF1B
:1041800080911F010E94E931AB01682F80912301CA
:104190000E94C30BF1CFDC011296ED91FC9142819C
:1041A000618180810C949B0C262FDC011296ED918D
:1041B000FC91428151816081822F0C94C30B089540
:1041C0000895FC01248130912302321B323360F0C8
:1041D0002E5C24830280F381E02D40E061818081A8
:1041E0000E94E9310C94150C08951F93CF93DF932F
:1041F000EC01EA81FB812E813F81418150E0809179
:10420000230290912402821B930B8417950708F4D4
:104210003EC0240F351F3F832E838C812D819081DA
:10422000182F299F1019112440E050E060E00E94EF
:10423000C10B0E94090C103430F440E050E060E003
:10424000812F0E94C10B8C819D81890F8C830E94DC
:10425000090C8C819D81190F803430F0292F219514
:104260002D83891B8C8310E440E050E06FEF8C813C
:104270000E94C10B0E94090C103448F44FEF50E02B
:1042800060E0812FDF91CF911F910C94C10BDF91E2
:10429000CF911F910895CF93DF93EC01EA81FB81C9
:1042A00090812F8180912302821B891700F1920F48
:1042B0009F83418150E0688570E08C819D810E94E0
:1042C00077319B01482F8E816C817D81860F972FDE
:1042D000911D8F3F910540F49D838C83842FB901FC
:1042E000DF91CF910C94150C8F5F9109F5CFDF9181
:1042F000CF9108951F93CF93DF93EC01EA81FB8167
:1043000080812F8190912302921B9817B8F1820F20
:104310008F8380917802811105C01092800281E024
:104320008093780210E02C813D811034F1F0912FC0
:104330009695969540E1949FC0011124820F931F9A
:104340008F3F910518F08F5F9109FACFEA81FB81C9
:10435000418150E0688570E00E947731AB01682FA1
:10436000812F0E94C10B1F5FDECF8E81820F932FA2
:10437000911D8F3F910530F49D838C83DF91CF9108
:104380001F9108958F5F9109F7CFFC016183089514
:10439000FC01618308954AE050E0682F85EF94E0C6
:1043A0000E94512C84E690E00E949B0460E285EF1D
:1043B00094E00E948C2B84E690E00C949B04809106
:1043C0000601882391F060E070E080E00E94150C07
:1043D0008091840290918502009739F0DC01ED9183
:1043E000FC910280F381E02D09940895CF93C82FAA
:1043F0008091B5049091B604892B51F460E370E08C
:104400008DE194E00E94EF139093B6048093B5047D
:1044100080E2C89FB00111248DE194E0CF910C940B
:10442000EF13CF93DF93EB019B0136952795820F16
:10443000931F0E94B636C0FF04C08F70DF91CF91EA
:1044400008958295FACFEF92FF920F931F93CF9327
:10445000DF9300D01F92CDB7DEB70091B504109165
:10446000B60493E0899F000D111D1124C8010E941C
:10447000B636F82EC80101960E94B636E82EC8015D
:1044800002960E94B63680958B83E094EA82F0947F
:10449000F98269817A818B810F900F900F90DF9163
:1044A000CF911F910F91FF90EF9008950E941122DC
:1044B0000C9423220F931F93CF93DF9320E2629FEC
:1044C00080011124080F191FD0E0C0E0BE01C8010F
:1044D0000E945622AB01682F8C2F0E94C10B21969F
:1044E000C034D10599F7DF91CF911F910F910895B5
:1044F000CF93C42F20E2629FB0011124860F971F33
:104500006FEF403428F4E42FF0E0EF52FD4F649158
:1045100070E00E945622AB01682F8C2FCF910C9433
:10452000C30BEF92FF920F931F93CF93DF9300D0B3
:1045300000D01F92CDB7DEB74B835C836D83FD80C7
:10454000F094EC80E0946B8160950091B50410913B
:10455000B60493E0899F000D111D11241A8309836D
:10456000CE0101960E948813C80101969A8389831F
:104570006E2DCE0101960E9488130E5F1F4F1A8385
:1045800009836F2DCE0101960E9488130F900F9022
:104590000F900F900F90DF91CF911F910F91FF908F
:1045A000EF9008951F93CF93DF93EB018CE294E09B
:1045B0000E94D717882379F067E176E085EF94E0D1
:1045C0000E94972B84E690E00E949B0480E0DF919C
:1045D000CF911F91089547E156E0BE018CE294E02F
:1045E0000E942E18882391F38CE294E00E943B18DD
:1045F000C0E0882391F08C2F0E942322D62F172F02
:104600000E94CB21812F0E94CB218D2F0E94CB2194
:10461000CF5FC03181F781E0DACF8CE294E00E9475
:104620003B18811120C041E070E060E085EF94E02C
:104630000E94C62CD62F41E070E060E085EF94E048
:104640000E94C62C162F41E070E060E085EF94E0F8
:104650000E94C62C462F512F6D2F8C2F0E94912225
:10466000CF5FC031D1F60E94DF21D5CF8F929F92CC
:10467000AF92BF92CF92DF92EF92FF920F931F9370
:10468000CF93DF9300D0CDB7DEB77B014A0159014C
:104690008CE294E00E94D7178823C9F0B40185EF1B
:1046A00094E00E94972B84E690E00E949B0480E0B7
:1046B0000F900F90DF91CF911F910F91FF90EF908E
:1046C000DF90CF90BF90AF909F908F900895A401FE
:1046D000B7018CE294E00E942E18882341F380E217
:1046E000089F600111248CE294E00E943B18F12C99
:1046F000E12C882341F1EC14FD0409F44EC0C701FC
:104700008A0D9B1D0E94B636082F10E082958F708F
:104710000E94CB21B8016F704AE050E085EF94E031
:104720000E943D2C84E690E00E949B0460E285EFAD
:1047300094E00E948C2B84E690E00E949B048FEF13
:10474000E81AF80AD8CF8CE294E00E943B18811155
:1047500022C0EC14FD04F9F041E070E060E085EF68
:1047600094E00E94C62C162F41E070E060E085EFD7
:1047700094E00E94C62CC7018A0D9B1D9A838983F1
:104780001295107F610FCE0101960E9488138FEF62
:10479000E81AF80AD8CF0E94DF2181E089CFE091A2
:1047A0000401F0E0E959FD4F80810E94BD0B809328
:1047B000B7049091B804981738F0682F8091B90425
:1047C0009091BA040C945A220895462F6091B70430
:1047D0009091B804961730F08091B9049091BA0482
:1047E0000C94782208958091B9049091BA04892B91
:1047F00049F4862F6093B8040E94F6219093BA047E
:104800008093B90408956CE276E085EF94E00E940D
:10481000682B84E690E00E949B0485EF94E00E9460
:10482000932B84E690E00E949B0480E00895FC01B5
:10483000908180910701981306C080918402909125
:1048400085020E94CF2380E008950F932091B90440
:104850003091BA040091B8044FE156E084EB94E043
:104860000E9436230F9108950E94B3110E94FA10FE
:10487000811104C00E94B3110C949B1184EC93E04D
:104880000E940C1386EA93E00C94F511803438F4FE
:10489000E82FF0E0EF52FD4F84910C94AE0D8FEFB6
:1048A000FCCF0E94B3110E94FA10811104C00E9433
:1048B000B3110C94001184EC93E00E94581286EA24
:1048C00093E00C9408128093BB0408950E94320E6A
:1048D0008091BB0481500E94ED0E8823B9F3809132
:1048E000BB0481500E940E0F8111F0CF08950E94E9
:1048F000150C0E94CE0B0C946624CF92DF92EF929F
:10490000CF93DF93C0904601D0904701E0904801DB
:10491000DEEFC0E04FEF50E06FEF70E08C2F90E0E3
:104920000E947731CF5FCF3F09F4C0E00E94150CA1
:104930000E94CE0BD15071F78E2DB6010E947724C4
:104940006FEF70E080E00E94772460E07FEF80E00E
:104950000E94772460E070E08FEFDF91CF91EF90BD
:10496000DF90CF900C947724CF93DF93CDB7DEB751
:10497000C054D1090FB6F894DEBF0FBECDBFCE0133
:1049800001966C0180E4F60111928A95E9F7609036
:10499000490170904A0180904B010E94320E10E054
:1049A00000E0F02E0034110509F454C0802F0E945D
:1049B000ED0E8823A1F0802F0E940E0F81110FC0F1
:1049C000F601E00FF11F808182608083883720F13B
:1049D000F601E00FF11F80818370808309C0F6012A
:1049E000E00FF11F8081982F969596959E31B8F033
:1049F0008F2D0E94ED0E811118C0F601E00FF11FFE
:104A0000808180FF1BC040E050E069EC8F2D0E9448
:104A100046240F5F1F4FC5CF81608083D9CF9F5F32
:104A2000990F990F8370892BD8CF8F2D0E940E0F6D
:104A300040E059EC882309F360E0E8CF682DA3013A
:104A400081FFE4CF8F2D0E94ED0E8111E2CF49EC62
:104A500050E0F2CF0E94CE0BA0CF0E9434240E94DF
:104A600051240E94500F0E947D240E94B42482E5AC
:104A700095E00E946D319091BD04882371F09111F1
:104A800009C081E08093BD0490E080E00E949F0512
:104A900080E0089581E090E0F9CF9923C9F3109266
:104AA000BD0482E090E0F2CF6BE376E085EF94E026
:104AB0000E94682B84E690E00E949B0485EF94E0BE
:104AC0000E94932B84E690E00E949B0480E008956E
:104AD0008F929F92AF92BF92CF92DF92EF92FF920E
:104AE0000F931F93CF93DF936C0110E000915B0154
:104AF000101708F04AC088E0189FE0011124F12C3B
:104B0000E12CFE01EC51FF4F5F018E2CF501EE0D03
:104B1000FF1D84918823B1F181500E94ED0E982EE3
:104B2000882349F0FFEFEF1AFF0A85E0E816F10449
:104B300061F785E0882E0E942F0F881221C09920EE
:104B4000F9F08091230290912402F60120813181B5
:104B5000821B930B20913101309132018217930710
:104B600078F0FE01EE51FF4F25913491812FF9012C
:104B700009958091230290912402F601918380830C
:104B80001F5FB6CF99249394D6CF80E0DF91CF9169
:104B90001F910F91FF90EF90DF90CF90BF90AF905B
:104BA0009F908F90089566E476E085EF94E00E94F0
:104BB000682B84E690E00E949B0485EF94E00E94BD
:104BC000932B84E690E00E949B0480E00895FC0112
:104BD000872F90E0982F8827680F792F711D6131FA
:104BE00080EC7807E0F0623188EC780750F461518E
:104BF000704C66A717A611AA80EE870F80AB81E0E4
:104C00000895633180ED780750F46251784C66A7BF
:104C100017A68AE2870F80AB84E481ABF0CF80E0F7
:104C200008958F929F92AF92BF92CF92DF92EF92B0
:104C3000FF920F931F93CF93DF9300D000D0CDB797
:104C4000DEB78C01F62E2FE3261708F469C0E62F95
:104C5000F0E0EE0FFF1FE35AFA4FD080E1808FEFB4
:104C6000D8120FC0E8120DC0AF2DB0E0A85DBD4F47
:104C7000E0910201F09103016F2D8C910995D82EDE
:104C8000E92E6D2D7E2DC8010E94E725B82E8111D9
:104C900035C0EF2DF0E0E85DFD4F8080C12CAA24E7
:104CA000AA94912CF8018281C81608F042C0F4E061
:104CB000CF9EC0011124F80160817181680F791FB6
:104CC000AA8244E050E0CE0101960E947C368981A0
:104CD0009A813B812C81F9122AC0482F082E000CA2
:104CE000550B4815590511F08F3F09F5F801D6A667
:104CF000E7A6C90190AB21ABBB24B3948B2D0F90D9
:104D00000F900F900F90DF91CF911F910F91FF9017
:104D1000EF90DF90CF90BF90AF909F908F900895CD
:104D20001092DD051092DE05EDEDF5E096CFC3940F
:104D3000B9CFD6A6E7A68FEF80AB81ABDFCFCF93FD
:104D4000DF93FC01EB019A01261B370BA4E6B0E0D0
:104D50000E94483626A130E050E040E00E9418361C
:104D60008091230290912402BC016C1B7D0B81E099
:104D70006217730708F080E0DF91CF910895292F23
:104D8000207C29F4805E883058F481E00CC0943493
:104D900039F496ED980F81E09A3228F080E008957A
:104DA00081E09634D9F70895CF93DF93EC018881A1
:104DB000681780F5882371F181508883E62FF0E031
:104DC000DF011196AC0FBD1FEE0FFF1F7196EC0FA8
:104DD000FD1F962F981780F411962C9111972D9303
:104DE00018962C91189717962C9317972281338138
:104DF000219331939F5FEECF2FEF30E001C0220F60
:104E00006A95EAF789A1922F909598238695822337
:104E1000892B89A3DF91CF910895CF93DF9300D0A1
:104E200000D01F92CDB7DEB7FC01348584A1982F46
:104E3000917080FD28C082E0248139838A836B834E
:104E40007C832D8391110AC0872F90E0982F8827AB
:104E5000680F792F711D64307105F0F460E0CF01A7
:104E600003960E94D42629813A814B815C816D8111
:104E700082E292E00F900F900F900F900F90DF91D1
:104E8000CF910C94F30981E0D7CF6D32710530F3E7
:104E90006933710518F703C068327105B0F784896A
:104EA000958994A783A7DACFCF93DF93FC01738111
:104EB000DC011D9681E090E060E08717F0F452A9D4
:104EC0004D9124A130E0082E02C0359527950A9413
:104ED000E2F720FD0DC0541721F080E0DF91CF9163
:104EE00008952489358934AB23AB682F0196E5CF2B
:104EF0005413FCCF8FEF82ABF0CF809123029091BF
:104F0000240223A934A9821B930B25A9281719066B
:104F100009F068F48FEF82AB6623F9F2EF01239674
:104F2000CE010E94D42660E0CE010E94D42681E00A
:104F3000D5CF7F928F929F92AF92BF92CF92DF9206
:104F4000EF92FF920F931F93CF93DF93EC019B811E
:104F5000911110C0F12C8F2DDF91CF911F910F91E6
:104F6000FF90EF90DF90CF90BF90AF909F908F9089
:104F70007F9008959C848CA180FF13C0983041F4E9
:104F800060E070E0CE010E940D27FF24F394E3CF90
:104F90008AA99812F5CFCE010E9454278111DACF49
:104FA000EFCF692DCE010E941126882309F470C02D
:104FB000FDA0FF2009F46CC00EA51FA5C8010E942A
:104FC000BF26882E80912302909124022BA53CA518
:104FD000821B930B2AA52817190609F010F57B8070
:104FE000A0902302B09024026E0101E010E0E12CB9
:104FF000202F071508F065C08CA190E0002E02C09C
:10500000959587950A94E2F780FD12C0811040C003
:10501000EE2009F454C07FEFC71AD70A0F5F1F4F65
:10502000E7CF8110DCCFB801CE010E940D27D7CF8A
:10503000F6019585FE013D9681E099122DC0EE2086
:1050400019F08EA1811110C0882059F068A979A9A2
:105050009AAA8C899D899CAB8BABCE010E940D27AF
:105060007ACF6EA57FA5F4CFF801EE0FFF1FEC0FEE
:10507000FD1F44895589EE2DF0E0EE0FFF1FEC0F68
:10508000FD1F64897589CE010E949F268111C3CFBF
:105090006EA57FA577CF8F5F821708F0BCCF3191C7
:1050A0003913F9CF4C895D89B501641B750B39A59E
:1050B0003617170609F078F768A979A9CECFE02E40
:1050C000AACF88E0781246CFE3CF0F931F93CF93F8
:1050D000DF93EC01FB0184819DA5282F291B12166B
:1050E0002CF09B8191111CC080E01FC08DA7808196
:1050F0008034D0F7818187FDF7CF8B018DA181119D
:1051000019C062817381CE010E94E725882361F373
:105110008EA59FA5D80113969C938E931297E4CFEA
:105120009C81891B87FDE0CF82E0DF91CF911F91A9
:105130000F9108952B81822F90E03481FE01E80FBA
:10514000F91F3483DB013C913487880F991FFE01DE
:10515000E80FF91F8091230290912402958B848B94
:1051600011964C913CA181E090E0A0E0B0E0022ECD
:1051700004C0880F991FAA1FBB1F0A94D2F740FFD3
:105180000CC041FD0AC0832B8CA32F5F2B83CE0163
:105190000E9499278111FBCFC7CF80958323F4CF3D
:1051A0000F931F93CF93DF93EC0120912302309153
:1051B00024028AA590E04BA55CA5B901641B750B80
:1051C0006817790738F0A90141505109481B590B5C
:1051D0005CA74BA78B818823D9F08C899D89281BDC
:1051E000390B8FA198A52817390768F00EA51FA5C0
:1051F000C8010E94BF26B801811102C068A979A91F
:10520000CE010E940D27CE010E9499278111FBCF6C
:1052100080E0DF91CF911F910F910895CF93DF939D
:10522000CEEBD4E0198218821A821B8288E0ECE46B
:10523000F1E0AAECB4E001900D928A95E1F781E0EB
:105240008DA380E58EA38AEF90E098A78FA382E3D9
:1052500089A78BE48AA780E091E09CA78BA78FEFBA
:105260008DA78EA78FA788AB89AB8AAB88EC8DAB57
:10527000DF91CF910895CF930E94B3110E94FA104D
:10528000C1E08111C0E08091E00081608093E00086
:105290000E94B311FC01C2870E94B3116C2F0E94BF
:1052A000FD1068EE73E080E090E00E94620480915F
:1052B000E0008E7F8093E000CF910895CF93DF933D
:1052C0001F92CDB7DEB76983DC01ED91FC910280BE
:1052D000F381E02D41E050E0BE016F5F7F4F099503
:1052E0000F90DF91CF910895CF93DF93EC018C85E0
:1052F0009D8597FF05C082E00E942F2E9D878C8799
:105300008C859D85DF91CF91089583E00E94462E84
:1053100090E0089583E00C94B530FC018485958578
:1053200097FD06C082E00E94C92D90E00196089585
:1053300082E00E94C92D90E00895FC018485958546
:1053400097FD05C02FEF3FEF35872487089582E052
:105350000C942F2ECF93DF93EC0180913E01882394
:1053600031F083E00E94602E1816190634F081E0B7
:1053700090E09B838A8380E090E0DF91CF91089555
:10538000EEEFFFE72591349181E02B3F3C4D09F092
:1053900080E00895FC0190819E5F908342E450E09C
:1053A0006DE476E080E80C94112FFC0181819081FE
:1053B000913A61F4813209F083C047E050E067E33D
:1053C00071E080E00E94112F81E00895913209F090
:1053D00077C0833269F482819381B0E0A0E080934A
:1053E000330190933401A0933501B0933601ECCF93
:1053F000803239F467E070E087E391E00E94372F54
:10540000E3CF823209F7828180933E010E94C02956
:10541000E0E0F8E0882311F0EEEFFAE08091370148
:1054200090913801A0913901B0913A01803B9440AC
:10543000A105B105D9F480913E0180FD17C0EE3F72
:105440008AE0F80771F587E797E791838083809179
:1054500060008093450588E19BE00FB6F894A8951D
:10546000809360000FBE90936000AECF80819181E9
:105470008737974709F0A8CFA89580916000886189
:10548000809360008091450580936000EE3F8AE044
:10549000F80789F08091FE0A9091FF0A918380833A
:1054A00093CF808191818737980769F29093FF0AA3
:1054B0008093FE0AC8CF1092FF0A1092FE0A84CF92
:1054C00080E008952FEF3FEFFC0135872487089592
:1054D000E5EFF4E01382128288EE93E0A0E0B0E002
:1054E00084839583A683B78388EC91E0918380833E
:1054F0008FEF9FEF958784870895EF92FF920F9328
:105500001F93CF93DF937B01FC01C281D38110E015
:1055100000E0209791F0E881F9810280F381E02D8D
:10552000B701CE01099597FD06C0080F191F088421
:10553000D985C02DEECF0FEF1FEFC801DF91CF91BE
:105540001F910F91FF90EF9008950F931F93CF93AA
:10555000DF938B01FC01C281D381209771F0E88138
:10556000F9810480F581E02DB801CE0109950097FD
:1055700031F40884D985C02DF0CF90E080E0DF9130
:10558000CF911F910F9108950F931F93CF93DF93A6
:105590008B01FC01C281D381209771F0E881F981F0
:1055A0000680F781E02DB801CE010995080F111D85
:1055B0000884D985C02DF0CFF8011082DF91CF91FA
:1055C0001F910F9108950F931F93CF93DF938B013A
:1055D000FC01C281D381209771F0E881F9810190AB
:1055E000F081E02DB801CE010995811105C0088434
:1055F000D985C02DF0CF80E0DF91CF911F910F9121
:105600000895CF93DF93FC01DB01218114968C91E7
:105610001497820F9927991F08978CF5C281D3811F
:10562000209731F573836283908112969C93129731
:1056300013962C93139715968C911597890F808349
:1056400080E014969C9114978917E8F41696CD91F2
:10565000DC911797C80FD11D9881C181D0E0C15C42
:10566000DE4F988391819F5F91838F5FEACFEC013A
:10567000888599850097D9F7B987A887D5CF80E025
:10568000DF91CF91089581E0FBCF80914605811194
:105690000DC082E080934E0584E080934F05109208
:1056A00051051092500581E0809346058EE495E007
:1056B0000895FB0101900020E9F73197AF01461BE7
:1056C000570BDC01ED91FC910280F381E02D0994F0
:1056D000EF92FF920F931F93CF93DF938C017B0187
:1056E000D0E0C0E0F701EC0FFD1F6491662361F08C
:1056F000D801ED91FC910190F081E02DC801099550
:10570000892B11F02196EECFCE01DF91CF911F9121
:105710000F91FF90EF900895DC01ED91FC910190C5
:10572000F081E02D099466ED71E00C94592B0F93F4
:105730001F93CF93DF93EC010E94682B8C01CE0165
:105740000E94932B800F911FDF91CF911F910F919A
:1057500008958F929F92AF92BF92EF92FF920F9314
:105760001F93CF93DF93CDB7DEB7A1970FB6F89411
:10577000DEBF0FBECDBF7C01FA01CB0119A22230E2
:1057800008F42AE08E010F5D1F4F822E912CB12C60
:10579000A12CBF01A50194010E941836F901CA018C
:1057A0006A300CF5605DD8016E938D01232B242B9C
:1057B000252B79F790E080E0109721F0BD01C7011B
:1057C0000E94592BA1960FB6F894DEBF0FBECDBF35
:1057D000DF91CF911F910F91FF90EF90BF90AF900D
:1057E0009F908F900895695CDECFCF92DF92EF9209
:1057F000FF920F931F93CF93DF932115310581F40F
:10580000DC01ED91FC910190F081E02D642FDF919E
:10581000CF911F910F91FF90EF90DF90CF9009945F
:105820002A30310501F52AE077FF1DC06A017B01AE
:10583000EC016DE20E948C2B8C0144275527BA01A4
:105840004C195D096E097F092AE0CE010E94A92B3F
:10585000800F911FDF91CF911F910F91FF90EF90DB
:10586000DF90CF900895DF91CF911F910F91FF901E
:10587000EF90DF90CF900C94A92B9A01AB01770F9A
:10588000660B770B0C94F52B2115310541F4DC01E7
:10589000ED91FC910190F081E02D642F09940C941E
:1058A000A92B9A01462F50E070E060E00C94442C44
:1058B0009A01AB0170E060E00C94442C0F931F93AD
:1058C000CF93DF93EC010E943104688779878A8740
:1058D0009B87E881F9810484F585E02DCE01099547
:1058E00097FF15C00E943104088519852A853B85DC
:1058F000601B710B820B930B0C811D812E813F81EC
:10590000601771078207930720F38FEF9FEFDF91F6
:10591000CF911F910F910895FF920F931F93CF93F3
:10592000DF93EC018B01F42ECE010E945E2C97FDDB
:105930001DC08D329105D1F09C01205331092A30D0
:105940003105A0F0FF2019F08E32910579F0013079
:10595000110551F00230110589F48D30910571F077
:105960005CF40997029750F08FEF9FEFDF91CF9192
:105970001F910F91FF9008958097B1F7E881F98109
:105980000284F385E02DCE010995CECFBF92CF9250
:10599000DF92EF92FF920F931F93CF93DF938C01CF
:1059A000C42F40E00E948C2CFC01C12CD12C76012C
:1059B00097FD3EC0B12C0C2E000CDD0BCE17DF077F
:1059C000D9F0ED32F10509F43FC0CF01C0970A9735
:1059D00098F4AAE0B0E0A70196010E9457366F0143
:1059E000FF0FEE08FF08C60ED71EE81EF91E80E363
:1059F000C81AD108E108F108D801ED91FC910284A0
:105A0000F385E02DC8010995C8010E945E2CFC01B8
:105A1000C0970A9798F2CE17DF0781F2BB2041F0BA
:105A2000F094E094D094C094C11CD11CE11CF11CF2
:105A3000C701B601DF91CF911F910F91FF90EF90B9
:105A4000DF90CF90BF900895BB24B394D5CF409101
:105A50005505509156052091530530915405421734
:105A60005307B4F49091E8009570E1F39091E80049
:105A700092FD19C08093F1008091550590915605D3
:105A800001968F739927892B19F48EEF8093E80084
:105A900080915505909156050196909356058093F7
:105AA000550581E0089580E00895EF92FF920F93ED
:105AB0001F93CF93DF93F82E192FE62E042F81E04A
:105AC000860F880F0E94272D83E00E94272DCF2D5F
:105AD000D12FEC0EFD2EF11CCE15DF05B9F007FF1E
:105AE00013C0FE0184910E94272D182F80E00E9490
:105AF000272D812321968111EFCFDF91CF911F9127
:105B00000F91FF90EF9008958881EDCF81E0F5CF60
:105B10008091D70081608093D70080EA8093D8007D
:105B200089B5806189BD89B5826089BD09B400FEEF
:105B3000FDCF61E070E080E090E00E94620480911F
:105B4000D8008F7C80618093D8008091E000807FB6
:105B50008093E0000895CF93DF931F92CDB7DEB717
:105B60001982CE0101960E94CA290E94452BBE01CE
:105B70006F5F7F4F0E947D2A89810F90DF91CF91C7
:105B800008952FB7FC012083F89467706093E900B3
:105B90000895CF93DF931F92CDB7DEB7682FCE0164
:105BA00001960E94C12D8091F200811107C0909151
:105BB000E80092FF03C09BE69093E80099819FBFA5
:105BC0000F90DF91CF910895EF92FF920F931F9363
:105BD000CF93DF931F92CDB7DEB7909159059923EC
:105BE000D9F157FD39C08A017B01682FCE0101969A
:105BF0000E94C12D8091F20081110BC09091E800AC
:105C0000892F847092FF05C08BE68093E800809115
:105C1000F20090E0081719070CF4C801282FF701CB
:105C200044E6215030F040935A053091F100319311
:105C3000F8CF009739F02091F200211103C02BE634
:105C40002093E80029812FBF0F90DF91CF911F9102
:105C50000F91FF90EF9008958FEF9FEFF5CFCF93C7
:105C6000DF931F92CDB7DEB741E050E0BE016F5F1A
:105C70007F4F0E94E42D019731F4898190E00F90CD
:105C8000DF91CF9108958FEF9FEFF9CFCF93DF93FF
:105C90001F92CDB7DEB7682FCE0101960E94C12DAD
:105CA0009091E800892F807295FF04C09091F200D6
:105CB00080E4891B99819FBF0F90DF91CF91089558
:105CC0005F926F927F928F929F92AF92BF92CF928C
:105CD000DF92EF92FF920F931F93CF93DF931F9268
:105CE000CDB7DEB7982E6B01B42E052F80915905E4
:105CF000811113C08FEF9FEF0F90DF91CF911F9114
:105D00000F91FF90EF90DF90CF90BF90AF909F905A
:105D10008F907F906F905F9008958091570580FFDE
:105D200005C08091E00082608093E000EB2CF02EB3
:105D3000A12C8AEF882E892D8072682E892D80747F
:105D4000582E9AE3792EE114F10419F4AA2009F4EB
:105D500057C0892D0E94462E182F81110AC08A949F
:105D6000882041F261E070E080E090E00E946204EF
:105D7000EACF8E151F0411F00CF01E2D692DCE01F7
:105D800001960E94C12D8091E80085FD03C08981A4
:105D90008FBFD9CF812F90E0E81AF90A662029F049
:105DA0001150A0F01092F100FBCFF60197FC0AC051
:105DB000115050F021912093F100FACF24912093BB
:105DC000F10031961150D0F7C80ED91EAA2021F04B
:105DD0007092E800A12CDBCF8091E80085FD08C01F
:105DE0007092E800AA24A394E114F10481F2F2CFA6
:105DF000E114F10461F6552051F27092E800C7CF2A
:105E000084E680935B058B2D902F76CF1092E9006E
:105E100010925605109255059093540580935305A2
:105E20000895DF92EF92FF920F931F93CF93DF932A
:105E3000D82E8A01EB017B01E40EF51ECE15DF059D
:105E400059F0D7FE12C0FE0184910E94272D2196A1
:105E50008111F4CF0FEF1FEFC801DF91CF911F9198
:105E60000F91FF90EF90DF9008958881EECFCF9350
:105E7000DF93EC019B01B4E6ABEF21153105F1F0A6
:105E8000A9012134310514F040E450E08091E8008C
:105E900082FFFCCF942FFB01E21BF30BEC0FFD1FE5
:105EA000915028F08091F10080833196F9CFB09322
:105EB0005A05A093E800241B350BDFCFCB01DF91FF
:105EC000CF9108951F920F920FB60F921124CF9287
:105ED000DF92FF920F931F932F933F934F935F9304
:105EE0006F937F938F939F93AF93BF93EF93FF93A2
:105EF000CF93DF93CDB7DEB76C97DEBFCDBF1092E7
:105F0000E9008091E80083FF2FC089E0FE017596CB
:105F1000FE2E0F2F815029F09091F1009083319641
:105F2000F9CF84E680935A0582EF8093E8008D894B
:105F300087FF38C09091E80090FFFCCF982F9076B3
:105F400009F000C19E894F89588D2F89188D9111B4
:105F500030C0803859F5809158058093F100109237
:105F6000F1008EEF8093E8006C960FB6F894DEBFD8
:105F70000FBECDBFDF91CF91FF91EF91BF91AF9158
:105F80009F918F917F916F915F914F913F912F9151
:105F90001F910F91FF90DF90CF900F900FBE0F9049
:105FA0001F9018959EEF9093E800C8CF1092F100D3
:105FB000D6CF913059F48111D4CF4130510589F6B3
:105FC000809158058D7F80935805CBCF933049F44D
:105FD0008111C7CF4130510521F68091580582606B
:105FE000F2CF953041F48091E80080FFFCCF20682B
:105FF0002093E300B6CF963009F076C0CB8CDC8CD2
:10600000123039F590E080E00E94062F0E94AB2DFF
:106010001F8299E099831A8391E09E8390EA988782
:106020009AEF99872091550530915605275F3F4F8C
:106030003C832B838D83C6010E94062F49E050E0EC
:10604000BE016F5F7F4F80E00E94112F0E94AB2D39
:1060500088CFC6010E94062F0E94452B6F2D702FFE
:106060000E94A52A009731F00CF07BCF81E280934B
:10607000EB007ACF113061F11330C1F78F8988239B
:1060800081F1823049F440E868E08CEA96E00E94B1
:10609000552D882359F365CF813029F440E86AE013
:1060A00081EA96E0F4CF833009F70E94452B8E01F8
:1060B0000F5F1F4FB8010E94C42AF8010190002011
:1060C000E9F73197BF01601B710B40E0C801DFCFDA
:1060D0006FE876E0FB01449150E080E80E94112FC8
:1060E00040CF65EB76E0F6CF973009F4BFCF98301C
:1060F00021F481E08093F10034CF993009F031CF61
:10610000837009F0B3CFE0E4F1E081E031E096E3A1
:106110002191222371F08093E9003093EB00DF019D
:1061200011972C912093EC009093ED008F5F8730B6
:1061300079F78EE78093EA001092EA008F898093C6
:1061400059050FCF8B8D9C8D0E94062F898D811153
:1061500005C08F2D902F0E94D5299BCF0E94452BE3
:106160006F2D702F0E94E32A94CF8093E9008091D5
:10617000F200882319F08AE38093E80008951F92C3
:106180000F920FB60F9211242F933F934F935F936B
:106190006F937F938F939F93AF93BF93CF93EF931F
:1061A000FF93C091E1008091E100837F8093E10043
:1061B000C3FF0FC01092E90081E08093EB001092C2
:1061C000EC0082E38093ED001092590588E0809303
:1061D000F000C2FF15C083E00E94B53080915B05DE
:1061E000882329F080915B05815080935B05809125
:1061F0005A05882329F080915A05815080935A05C9
:10620000C4FF23C08091E2008E7E81608093E20013
:106210008091E1008F7E8093E100809157058E7E12
:10622000806180935705FF91EF91CF91BF91AF911E
:106230009F918F917F916F915F914F913F912F919E
:106240000F900FBE0F901F901895C0FFECCF80915C
:10625000E2008E7E80618093E2008091E1008E7E7C
:106260008093E100809157058E7E8160DACF109295
:10627000590510925805109257050E94882DE1EE9D
:10628000F0E080818E7E80838DE08093E200559ADD
:10629000209A08959091590581E0911101C080E004
:1062A00008958091E0008D7F8093E0008091E00070
:1062B00081FD11C08091570580FF0DC08091580568
:1062C00081FF09C00E94882D8091E0008260809348
:1062D000E00081E0089580E0089580915705817085
:1062E000089508951092DD051092DE0508950F932C
:1062F0001F93CF93DF93FB01742F309739F4642FF2
:10630000842FDF91CF911F910F91089566E0689FD0
:106310009001699F300D1124E901DD27CE9FD00146
:10632000CF9FB00DDE9FB00D1124AB2FBB278FEF99
:1063300090E08C010A1B1B0B049FD001059FB00D40
:10634000149FB00D11248C010C1B1D0B0E9FE0013E
:106350000F9FD00D1E9FD00D1124CD2FDD278C0156
:106360000C1B1D0B049FE001059FD00D149FD00D49
:1063700011248E1B9F0B849FF001859FF00D949F2D
:10638000F00D11246F2F232F332722303105F1F028
:1063900060F421153105B9F08B2F2130310509F456
:1063A000B0CF842F7F2F6B2FACCF8F2F642F7B2FFD
:1063B0002330310509F4A5CF8D2F7F2F24303105EF
:1063C00009F49FCFEECF842F7D2F9BCF8F2F6D2F82
:1063D00098CF90E1499FA001112420912302309190
:1063E0002402420F531FA4E056954795AA95E1F762
:1063F000942F47FD9095990F999FF0011124EF2F4D
:10640000FF27AF01440F551F4E0F5F1F9E9F900146
:106410009F9F300D1124232F3327220F331F421B40
:10642000530B56954795405B50E070E090E00C941C
:1064300077311092050681E08093030610920206E0
:10644000589A599AE9EBF0E080818E7F80838081B1
:106450008D7F808388E48093B80085E48093BC00BE
:106460000895413208F043C0909105069111FCCF88
:1064700091E090930506209303062FEF2093DF050C
:106480001092E105240F2093E0059093040690916B
:106490000406880F892B80930406809102068130C0
:1064A00009F510920206809104068093BB0080914A
:1064B000BC0083FDF8CF85EC8093BC00809105067D
:1064C0008130E1F38091E105841710F44091E105FA
:1064D000A2EEB5E0962FFB018E2F891B841720F0CA
:1064E000842F089585EEE8CF8D918193F5CF40E01C
:1064F000F7CF0F93413208F04BC0909105069111F0
:10650000FCCF92E090930506009303069FEF9093D3
:10651000DF051092E1054093E005362FA2EEB5E0CD
:10652000FB019E2F931B941750F11092040690913B
:106530000406880F892B809304068091020681301F
:1065400009F510920206809104068093BB008091A9
:10655000BC0083FDF8CF85EC8093BC00222321F0A2
:10656000809105068230D1F38091DF05803361F0A0
:106570008F3F81F0803251F482E00F910895919124
:106580009D93CFCF85EEE8CF83E0F7CF84E0F5CFC2
:1065900081E0F3CF80E0F1CF85ED8093BC00809166
:1065A000BC0084FDFCCF10920506089585EC809315
:1065B000BC001092050608951F920F920FB60F921D
:1065C00011242F933F934F935F936F937F938F93F8
:1065D0009F93AF93BF93EF93FF938091B900887F10
:1065E0008832F1F100F5803199F1B0F4882309F493
:1065F00075C0883069F1FF91EF91BF91AF919F9184
:106600008F917F916F915F914F913F912F910F905B
:106610000FBE0F901F901895883111F1803259F7F5
:106620008093DF0512C08034C1F148F48033C1F398
:10663000883309F78093DF050E94D632DCCF80359E
:1066400001F1883591F18834B1F60E94CC32D3CF74
:10665000809104068093BB0085EC8093BC00CBCF77
:106660009091E1058091E005981758F5E091E105DA
:1066700081E08E0F8093E105F0E0EE51FA4F8081CA
:10668000E9CFE091E10581E08E0F8093E1058091F3
:10669000BB00F0E0EE51FA4F80839091E1058091CC
:1066A000E0059817C8F285E8D8CFE091E10581E0D0
:1066B0008E0F8093E1058091BB00F0E0EE51FA4F20
:1066C0008083809103068111C0CF81E08093020610
:1066D00084EA8093BC00109205068DCF1092DF05EE
:1066E000B4CFCF93DF93CDB7DEB769970FB6F894E9
:1066F000DEBF0FBECDBFFC01DB018C918F5F8C93A1
:106700009E012D5F3F4F8DE0D9011D928A95E9F7DB
:1067100029E0298384E08A8391E09D8383E08E834E
:106720002A8721E22B879C879D879F8722E2288BDF
:1067300027E02B8B25E02C8B8E8B20E430E0388FEC
:106740002F8B998F82818B8395858685998B8A8BF8
:10675000838180688D8B49E150E0BE016F5F7F4F80
:1067600080E00E94112F69960FB6F894DEBF0FBE2D
:10677000CDBFDF91CF9108950F931F93CF93DF93F8
:10678000FB012081213879F52381223261F5DC017A
:1067900012964C91248135814217130621F5EC01A4
:1067A00081E00E9403360B84DC85C02D10E000E000
:1067B000209781F04C815D816A817B8180E80E9415
:1067C000112F8F3F980751F0080F191F0990D8819A
:1067D000C02DEECF80E00E940336C801DF91CF913B
:1067E0001F910F91089590E080E0F8CFCF93DF9351
:1067F000FC014281FB012481358142171306A1F57A
:10680000EC0181819081913A71F4813051F08230B4
:1068100059F5BE01605F7F4F41E050E080E40E9487
:10682000112F81E022C09132F9F48B30E9F08A30E7
:1068300019F48381888BF5CF8930B1F486819781F3
:106840008230910539F462E070E0CE0141960E94F9
:10685000372FE7CF019729F761E070E0CE0142962C
:106860000E94372F198ADDCF80E0DF91CF91089504
:10687000FC01A385B485109771F4748763878585BF
:106880009685DB0114962D913C91820F931F96877C
:1068900085870895DC018D919C9111970097D1F720
:1068A0006D937C93ECCFAF92BF92CF92DF92EF9239
:1068B000FF920F931F93CF93DF931F92CDB7DEB755
:1068C0007C0169836A01590141E050E0BE016F5FBC
:1068D0007F4FFC0183810E94602E8C0197FD0BC0CD
:1068E000F7018381A501B60180640E94602E080F24
:1068F000191F97FD8C01C8010F90DF91CF911F9157
:106900000F91FF90EF90DF90CF90BF90AF900895E0
:10691000CF92DF92EF92FF921F93CF93DF93162FC8
:106920007A0169010E945334EC01E091A403F091D3
:10693000A503309729F09C01A601B701812F099585
:10694000CE01DF91CF911F91FF90EF90DF90CF901C
:106950000895CF93DF93EC0181E08C838D839E01BA
:10696000265F3F4F3F832E83198618862DED31E039
:10697000398328831C861B861E861D868F87188A6E
:106980000E94B311198A1A8A81EC8A870E94452BCA
:10699000BE01DF91CF910C94012B809106068111ED
:1069A00007C08EE096E00E94A93481E0809306063D
:1069B0008EE096E00895FC011582809127068111F2
:1069C00013C01092300610922F0689EB96E0909338
:1069D0003206809331068FE390E0909334068093E3
:1069E000330681E0809327060E94CD346FE276E083
:1069F0000C9438340F93FC01618342832383048316
:106A00000F91089525E0FC0111922A95E9F7089568
:106A1000FC019081692B60830895CF93DF93EC0193
:106A20000E94CD3425E030E0AE0161E0DF91CF91EE
:106A30000C948834CF93DF93EC0198818D81981367
:106A40000CC08981811109C08A81811106C08B81A6
:106A5000811103C08C81882329F0CE010E940D355D
:106A600088818D83DF91CF91089581E296E00C9427
:106A7000DB34CF93DF93CDB7DEB769970FB6F894C9
:106A8000DEBF0FBECDBFFC01DB019C919F5F9C93DD
:106A90009E012D5F3F4F81E1D9011D928A95E9F753
:106AA00029E0298384E08A8391E09D8383E08E83BB
:106AB0002A8721E22B879C879D879F8722E2288B4C
:106AC0002AE3298B27E02B8B25E02C8B8E8B20E46F
:106AD00030E0388F2F8B998F82818B838381806800
:106AE0008D8B49E150E0BE016F5F7F4F80E00E94D7
:106AF000112F69960FB6F894DEBF0FBECDBFDF91A0
:106B0000CF9108950F931F93CF93DF93EB018A01E9
:106B1000FC01838180640E94602EE091A403F091C7
:106B2000A503309749F09C01A801BE0187E0DF91E1
:106B3000CF911F910F910994DF91CF911F910F91E8
:106B400008950A970C948235FB01DC0112964C9152
:106B5000248135814217130639F421813081313A7D
:106B600029F481E0213009F080E008953132E1F725
:106B70002A30D1F72281FC01238B81E00895FB01AB
:106B80002081213891F42381223279F4DC0112969C
:106B90002C91848195812817190639F44AE350E035
:106BA00068EF76E080E80C94112F90E080E0089583
:106BB000CF93DF93EC0181E08C838D839E012F5E68
:106BC0003F4F3F832E83198618861D861C861F869D
:106BD0001E86188A29EE31E03983288327EF31E0B9
:106BE0003B872A878A8B8B8B0E94B31181EC898B20
:106BF0000E94452BBE01DF91CF910C94012B85E3C0
:106C000096E00C94D8350895AA1BBB1B51E107C030
:106C1000AA1FBB1FA617B70710F0A61BB70B881F2C
:106C2000991F5A95A9F780959095BC01CD010895BB
:106C3000A1E21A2EAA1BBB1BFD010DC0AA1FBB1F80
:106C4000EE1FFF1FA217B307E407F50720F0A21BF2
:106C5000B30BE40BF50B661F771F881F991F1A945F
:106C600069F760957095809590959B01AC01BD0189
:106C7000CF010895EE0FFF1F0590F491E02D0994C8
:106C80000E9462368F93CB010E9462360C94693663
:106C9000A29FB001B39FC001A39F700D811D11245D
:106CA000911DB29F700D811D1124911D08950E94A8
:106CB0004836A59F900DB49F900DA49F800D911D07
:106CC000112408950E946C368F93892F0E946C3690
:106CD00099270F90800D0895082E817006940694D0
:106CE000811D0694811D0694811D0694811D0694C4
:106CF000811D0694801D0895FB01DC0102C00590F2
:106D00000D9241505040D8F70895FB01DC018D9160
:106D1000059080190110D9F3990B0895FB01DC014E
:106D200004C08D910190801921F441505040C8F762
:106D3000881B990B0895FB01DC0102C001900D92A4
:106D400041505040D8F708956817790768F4FB015F
:106D5000DC01E40FF51FA40FB51F02C002900E92D4
:106D600041505040D8F708950C949B36F999FECFC6
:106D700092BD81BDF89A992780B50895262FF9997B
:106D8000FECF1FBA92BD81BD20BD0FB6F894FA9A0E
:0C6D9000F99A0FBE01960895F894FFCF09
:106D9C0003FF570A012001FFFF0101320132E80312
:106DAC000200000000000000FFAA0000A0F023AACF
:106DBC000043FFFFAAFF059628322832FF0000F49B
:106DCC0001F401FFFFFFFF00E100000000000000E4
:106DDC00C18081000000A0A0A00064C9FFFFFFFFDC
:106DEC00FFFFFFFF6B62696F30310002220200006F
:106DFC000000FC0CFE0CFD0C030D00000000420D0D
:106E0C000000000093102F107A10281000000000D2
:106E1C00FC0CCB20FD0CD42000000000FC0CDF206F
:106E2C00E120E02000000000FC0CDF20F520E02039
:106E3C0000000000FC0CDF204B21E02000000000D3
:106E4C00FC0CDF207A21E02000000000FC0CCF239A
:106E5C00FD0CE523000000005E29AA2985298A295A
:106E6C008D299D2974290D0A0000000000F633714C
:106E7C0033BC335C0500000000A4353935BF352820
:0A6E8C00108235F6FF0000A135006A
:00000001FF
